:020000040800F2
:10000000C08C0020BD010008C5010008C701000820
:10001000C9010008CB010008CD0100080000000064
:10002000000000000000000000000000CF010008F8
:10003000D101000800000000D3010008D50100082C
:10004000D7010008D7010008D7010008D701000830
:10005000D7010008D7010008D7010008D701000820
:10006000D7010008D7010008D7010008D701000810
:10007000D7010008D7010008793F0008D701000820
:10008000D7010008D7010008D701000800000000D0
:10009000000000000000000000000000D701000880
:1000A000D7010008D7010008D7010008D7010008D0
:1000B00021280008A12F0008D7010008D701000857
:1000C000D7010008D7010008D7010008D7010008B0
:1000D000D701000885400008D7010008DD45000869
:1000E000D7010008D7010008D70100080000000070
:1000F0000000000000000000000000000000000000
:1001000000000000000000000000000000000000EF
:100110000000000000000000D7010008D70100081F
:1001200000F002F800F03AF80AA090E8000C8244CF
:100130008344AAF10107DA4501D100F02FF8AFF2AC
:10014000090EBAE80F0013F0010F18BFFB1A43F0B5
:10015000010318470C4201002C420100103A24BF51
:1001600078C878C1FAD8520724BF30C830C144BF1C
:1001700004680C607047000000230024002500265E
:10018000103A28BF78C1FBD8520728BF30C148BFFA
:100190000B6070471FB51FBD10B510BD04F0E8FD22
:1001A0001146FFF7F7FF02F0A3F904F006FE03B4CF
:1001B000FFF7F2FF03BC04F007FE00000948804788
:1001C00009480047FEE7FEE7FEE7FEE7FEE7FEE739
:1001D000FEE7FEE7FEE7FEE704480549054A064B51
:1001E000704700003924000821010008C086002063
:1001F000C08C0020C0880020C08800202749084308
:10020000274908607047F0B50F21C47802780123B0
:100210004FF0E026DCB1224C2468457804F4E06419
:10022000C4F5E064240AC4F10407E1408478BD40C9
:100230000C402C4321011B4C1155007800F01F018C
:100240008B40400906EB8000C0F80031F0BD02F0A1
:100250001F008340500906EB8000C0F88031F0BDDC
:10026000114A114001430E48001F016070470C4ABB
:10027000121D0029116801D0014300E08143116083
:1002800070474FF0E0210428086903D020F00400F3
:100290000861704740F00400FAE700000000FA052A
:1002A0000CED00E000E400E080FFFF1FC54910B541
:1002B000884202D1012144150AE0C349884202D193
:1002C0000121041504E0C14988420AD10121CC036F
:1002D000204601F089F82046BDE81040002101F0D9
:1002E00083B810BD10B54268B94B0C791A400B6841
:1002F00042EA0422134343608368B64A1340D1E9BB
:10030000024222434C7943EA44031A438260C26AA0
:10031000097C22F47002491EC9B242EA0151C1624D
:1003200010BD00210160017141718160C160012136
:10033000017470470029816802D041F0010101E099
:1003400021F00101816070470029816802D041F4E9
:10035000807101E021F4807181607047002A426859
:10036000C9B201D00A4300E08A4342607047816805
:1003700041F0080181607047014600208968090743
:1003800000D501207047816841F004018160704709
:10039000014600208968490700D5012070470029DF
:1003A000816802D041F4A00101E021F4A001816044
:1003B0007047014600208968490200D50120704736
:1003C0004268491E22F4604242EA4131416070476E
:1003D0000029416802D041F4006101E021F400618C
:1003E0004160704770B5072409290AD9C568A1F191
:1003F0000A0606EB4606B440A543B3401D43C5605C
:1004000007E0056901EB4106B440A543B3401D4335
:1004100005611F23072A09D2446B521E02EB820298
:1004200093409C4391400C43446370BD0D2A09D214
:10043000046BD21F02EB820293409C4391400C4319
:10044000046370BDC46A0D3A02EB820293409C4380
:1004500091400C43C46270BD0029816802D041F410
:10046000801101E021F4801181607047C06C80B27E
:10047000704754484C30006870470029416802D0EA
:1004800041F4806101E021F48061416070470029FE
:10049000416802D041F4805101E021F48051416073
:1004A0007047826822F4E0420A4382607047002964
:1004B000816802D041F4004101E021F400418160F3
:1004C00070470029816802D041F4021101E021F453
:1004D000021181607047014600208968890200D5B9
:1004E0000120704770B5072409290AD9C568A1F110
:1004F0000A0606EB4606B440A543B3401D43C5605B
:1005000007E0056901EB4106B440A543B3401D4334
:100510000561836BC3F30154121B921C02EB82042E
:100520001F22A2409343A1400B43836370BD826BA3
:10053000491E22F4401242EA01518163704708B516
:1005400008440090026008BD08B5084428300090B7
:10055000006880B208BD42681F4B1A400A434260DF
:100560007047416282627047426822F01F020A436C
:1005700042607047134908310028086802D040F4EF
:10058000000001E020F400000860704702460020EF
:1005900012680A4200D001207047C94301607047C9
:1005A00010B50246002054680B0AC9B20C4011680D
:1005B000194202D0002C00D0012010BD6FEA112199
:1005C000016070470024014000280140003C0140C8
:1005D000FFFEF0FFFDF7F1FFFFFD3FFF10B501202B
:1005E00000F014FFBDE81040002000F00FBF1F49CD
:1005F000086070471D49091F086070471B49843116
:10060000086070471A4A118821F460710143118013
:100610007047174A118821F07F010143118070470C
:10062000134A08B52C3A10440090016008BD1049E7
:1006300008B52C3908440090008808BD0B489C3050
:100640000068C0B270470A480830018841F00101D3
:10065000018070470548A0300068C0B27047044868
:100660000830018841F002010180704704860D4284
:100670002C6C004010B501214C07204600F0BDFE57
:100680002046BDE81040002100F0B7BE30B5374C21
:10069000236840F6FE7282409343D1E900252A4345
:1006A000D1E902510D432A4382401A43226030BDF2
:1006B0000021016041608160C16070472B4A0123C5
:1006C0008340106809B1184300E0984310607047F8
:1006D000264A93148340106809B1184300E09843F8
:1006E00010607047214A121D03090120984000291B
:1006F000116801D0014300E08143116070471B493C
:10070000091D0028086802D040F0030001E020F035
:10071000030008607047154B814018680AB1084310
:1007200000E0884318607047104A08B5104408304C
:100730000090016008BD0D4A08B5104414300090C7
:10074000016008BD082805D042EA0141074A10446B
:100750000162704742EA0121F8E7044908B501EB5C
:1007600090002C300090006880B208BD00740040FA
:1007700001684FF6FE721140016000210160416086
:100780008160C1606A496A4A0839904203D1486869
:1007900040F00F0006E0664A1432904204D14868E7
:1007A00040F0F00048607047614A2832904203D11F
:1007B000486840F47060F5E75D4A3C32904203D1EE
:1007C000486840F47040EDE7594A5032904203D1F6
:1007D000486840F47020E5E7554A6432904203D1FE
:1007E000486840F47000DDE7514A7832904203D106
:1007F000486840F07060D5E74E4A111F904203D11F
:10080000086840F00F0006E04A4A1432904204D1D2
:10081000086840F0F00008607047464A283290426D
:1008200003D1086840F47060F5E7424A3C329042D8
:1008300003D1086840F47040EDE73E4A50329042E0
:10084000EAD1086840F47020E5E730B5036847F660
:10085000F07293430C6A8A682243D1E904452C4321
:1008600022438C692243CC6922434C6A22438C6A1E
:1008700022431A430260CA6842600A68826049687B
:10088000C16030BD0021016041608160C1600161D3
:1008900041618161C16101624162816270470029E9
:1008A000016802D041F0010102E04FF6FE721140F2
:1008B00001607047002A026801D00A4300E08A43C1
:1008C0000260704741607047406880B270470146DF
:1008D0000020CA0002D5174A083A01E0144A083A33
:1008E00012680A4200D001207047C10003D51149A7
:1008F000091F086070470E49083948607047014673
:100900000020CA0002D50B4A083A01E0084A083A1A
:1009100012680A4200D001207047C10003D5054982
:10092000091F086070470249083948607047000095
:100930000800024008040240374900200860091DF1
:100940000860091D0860091D0860334933481431E7
:100950000860704730B530498379026853B30B683B
:1009600093430B600A1D13680468A3431360027964
:100970000A441368046823431360274A0832136843
:100980000468A3431360131D1C680568AC431C6016
:100990004479102C05D021440A68006802430A609B
:1009A00030BD116804682143116019680068014373
:1009B000196030BD0079084401689143016030BD81
:1009C0000021016001710C2242718171704712494E
:1009D00010310A6802430A60704701460E4A00203F
:1009E000143212680A4200D0012070470A491431BB
:1009F00008607047084A014600201268064B0A400A
:100A000014331B680B4202D0002A00D0012070472B
:100A1000014914310860704700040140FFFF0F00D6
:100A2000FC4A116801F03801014311607047F9492F
:100A30000A6822F008020A600A6802430A607047E6
:100A4000F4490A6822F010020A600A6802430A6048
:100A50007047F048F0494160F04941607047ED4807
:100A6000ED494160ED4941607047EA48016941F054
:100A7000800101617047E748016941F0800101612F
:100A80007047E4490420CA68D20701D001207047AA
:100A9000CA68520701D502207047C968C906FBD54C
:100AA0000320704700B50346FFF7EBFF03E000BFEC
:100AB000FFF7E7FF5B1E012803D0002B00D10520C4
:100AC00000BD002BF4D1FAE770B505464FF430268F
:100AD0003046FFF7E7FF042811D1CE4C206940F0E3
:100AE000020020616561206940F0400020613046CD
:100AF000FFF7D8FF216941F6FD721140216170BDF9
:100B000030B54FF430252846FFF7CCFF042810D12C
:100B1000C04C206940F004002061206940F0400092
:100B200020612846FFF7BEFF216941F6FB721140A4
:100B3000216130BD00B50346FFF7A3FF03E000BF0E
:100B4000FFF79FFF5B1E012803D0002B00D105207B
:100B500000BD002BF4D1FAE730B54FF4302528461C
:100B6000FFF7E8FF042810D1AA4C206940F00400E8
:100B70002061206940F0400020612846FFF7DAFF3D
:100B8000216941F6FB721140216130BDA14900206D
:100B9000C969890700D50120704770B5A525FFF701
:100BA000F5FF00B100254FF430263046FFF77AFFFD
:100BB000042827D1974C9848A0609848A0602069E5
:100BC00040F020002061206940F040002061304664
:100BD000FFF768FF41F6EF7604280ED1206941F651
:100BE000DF7108402061206940F0100020618C48CE
:100BF00005804FF40050FFF755FF052802D021690A
:100C00003140216170BDF8B5064600204FF4005C0C
:100C100000900D466046FFF745FF042816D17D4C35
:100C2000206940F00100206135806046FFF73AFFFF
:100C300041F6FE77042806D1B61C280C00963080B9
:100C40006046FFF72FFF216939402161F8BDF0B5FB
:100C500006464FF400570D463846FFF723FF042899
:100C60000CD16C4C206940F0010020613580384681
:100C7000FFF718FF2169BA1E11402161F0BDF0B5E0
:100C800006464FF400570D463846FFF70BFF042881
:100C900013D1604C6048A0606048A060206940F0BB
:100CA0001000206135803846FFF7FCFE052804D08F
:100CB000216941F6EF7211402161F0BD2DE9F0414B
:100CC000C04300F0FF0CC0F30727C0F30746050E32
:100CD0004FF400584046FFF7E5FE042837D14D4C4D
:100CE0004D49A1604D49A160216941F01001216188
:100CF000BCF1FF0F08D04A480830A0F800C04046B9
:100D0000FFF7D0FE04281BD1FF2F07D044480A303C
:100D100007804046FFF7C6FE042811D1FF2E07D0FA
:100D20003F480C3006804046FFF7BCFE042807D140
:100D3000FF2D07D03A480E3005804046FFF7B2FE3F
:100D4000052804D0216941F6EF7211402161BDE808
:100D5000F08170B505464FF430263046FFF7A2FE0D
:100D6000042818D12B4C2C48A0602C48A060206986
:100D700040F020002061206940F0400020613046B2
:100D8000FFF790FE41F6DF71042805D0052802D058
:100D900022690A40226170BD2069084020612069F3
:100DA00040F0100020611E480DB1002100E0A52197
:100DB00001803046FFF776FE0528ECD0216941F628
:100DC000EF721140216170BDF0B5124C0746124818
:100DD00016460D46A0601148A0604FF4005C6046C6
:100DE000FFF760FE042814D1206940F01000206154
:100DF00035430B493D43891C45F0F80008806046A7
:100E0000FFF750FE052804D0216941F6EF7211402A
:100E10002161F0BD0020024023016745AB89EFCD81
:100E200000F8FF1F1C48C069800870471A48006A14
:100E30007047194900200968890600D501207047CC
:100E4000154A0029116901D0014300E08143116175
:100E5000704701460020104A012903D0D2680A4297
:100E600003D17047D169C907FBD0012070470A49F7
:100E7000C860704708490420CA68D20701D0012021
:100E80007047CA68520701D502207047C968C90671
:100E9000FBD5032070470000002002408F4910B5A9
:100EA000884206D10121042000F09EFA002104208E
:100EB0003BE08B49884206D10121082000F094FADA
:100EC0000021082031E08749884206D10121102005
:100ED00000F08AFA0021102027E08349884206D1D9
:100EE0000121202000F080FA002120201DE07F4910
:100EF000884206D10121402000F076FA00214020EE
:100F000013E07B49884206D10121802000F06CFA71
:100F10000021802009E0774988420AD18415012107
:100F2000204600F061FA00212046BDE8104000F0A4
:100F30005BBA10BD10B50121084600F055FA00213A
:100F4000BDE81040012000F04FBAF0B5CA78002586
:100F500002F00F03D20601D58A7813430C784FF0C4
:100F60000F0E0122E4B104680F8802FA05F637403B
:100F7000B74211D14FEA850C0EFA0CF724EA0707A5
:100F800003FA0CF43C43CF78282F02D0482F02D02C
:100F900002E0466100E006616D1C082DE4D30460A8
:100FA0000C88FF2C1ED944685FF0000606F1080784
:100FB00002FA07F50F882F40AF420FD14FEA860C97
:100FC0000EFA0CF7BC4303FA0CF73C43CF78282FFA
:100FD00000D14561CF78482F00D10561761C082EDD
:100FE000E4D34460F0BD4FF6FF71018002218170AF
:100FF0000421C17070470246002092680A4200D066
:1010000001207047806880B2704702460020D26895
:101010000A4200D001207047C06880B27047016169
:101020007047416170470AB1016170474161704783
:10103000C160704741F4803282618161826181695F
:10104000806970472C4B10B51A684FF680742240A7
:1010500042EA00100843186010BD2849C861704773
:10106000F0B5254C002801DAE36900E06368420D21
:10107000120185B2C0F301579540C0F30346032F18
:1010800005D0C2020AD50322B240934307E023F001
:101090007062636823F07063636002E0AB4343F007
:1010A000706201B12A43002801DAE261F0BD62609A
:1010B000F0BD10B58A0721F003040F49130F214436
:1010C0000F228C689A4094438C608A68984002434F
:1010D0008A6010BD0949DC31086070470008014092
:1010E000000C0140001001400014014000180140B4
:1010F000001C01400020014000000140000020428F
:1011000010B501210C07204600F077F92046BDE814
:101110001040002100F071B9214908627047204950
:10112000086170471F4A116821F0E0010143116016
:1011300070471B49A031086070471A4B1A6822F0AB
:10114000030202431A601848026842F00402026077
:10115000012905D020BF016821F00401016070471A
:1011600030BFF8E70F48016841F0040101600168F1
:1011700041F0020101600C48016841F00401016086
:1011800030BF7047074A0146002052680A4200D02B
:101190000120704703490A6842EA800008607047EE
:1011A00000000E420070004010ED00E0A54801680C
:1011B00041F0010101604168A34A114041600168AA
:1011C000A24A11400160016821F480210160416858
:1011D00021F4FE0141604FF41F018160704799497D
:1011E0000A6822F480320A600A6822F480220A60C7
:1011F000B0F5803F07D0B0F5802F03D1086840F4E8
:10120000A02008607047086840F48030F9E7024683
:10121000002053098B49012B0AD0022B0AD0496ABE
:1012200002F01F02012393400B4200D001207047BF
:101230000968F5E7096AF3E718B500204FF4A064E0
:1012400000903120FFF7E3FF0099491C0091A14273
:1012500001D00028F5D03120FFF7D9FF002800D0B9
:10126000012018BD77490A6822F0F80242EAC0005E
:1012700008607047764908607047724A53680843AF
:1012800023F47C1318435060704771490866704717
:101290006C4A516821F0030101435160704769486D
:1012A000406800F00C007047664A516821F0F00178
:1012B000014351607047634A516821F4E061014382
:1012C000516070475F494A6822F4605242EAC000A8
:1012D000486070475B4A0029517A01D0014300E021
:1012E0008143517270475A49D83108607047554A56
:1012F000516821F440410143516070475149002237
:1013000081F8202081F82020012802D0042802D171
:10131000052081F8200070474E4908607047494910
:101320000A6A02430A6270474A49443908607047B2
:1013300030B544494A6812F00C03474A03D0042BE5
:1013400001D0082B22D002604A680F23434C03EAE5
:101350001212A35C0268DA4042604B68072505EA76
:101360001323E35C22FA03F383604B6805EAD3237B
:10137000E35C22FA03F2C2604968032303EA913175
:10138000231F595CB2FBF1F1016130BD4A684B6823
:1013900002F470124FF0020413F4803F04EB924207
:1013A00002D04B689B0301D52D4B00E02A4B5A43DA
:1013B000C9E7244A0029516901D0014300E0814373
:1013C000516170471F4A0029916901D0014300E033
:1013D0008143916170471B4A0029D16901D00143C3
:1013E00000E08143D1617047164A0029D16801D0DD
:1013F000014300E08143D1607047124A002911691E
:1014000001D0014300E08143116170471149403927
:10141000086070470E49C86470470A49C871704730
:101420000848416A41F0807141627047054A0146AF
:10143000002092680A4200D001207047014988725A
:1014400070470000001002400000FFF8FFFFF6FEAA
:10145000000042428004424200127A000400002050
:1014600000093D00424A0029118801D0014300E0F3
:101470008143118070473E48001D018841F01001F2
:10148000018070473A48001D018821F01001018059
:10149000704737481C30008835491831098840EAC0
:1014A0000140704700B50246FFF7E5FF3049100CD8
:1014B00018310880081D02805DF804EBE2E700B5F2
:1014C0000246FFF7D8FF2A49C2F3034008310880DB
:1014D000081D02805DF804EBD4E700B50246FFF773
:1014E000CAFF2349100C20310880081D02805DF8D6
:1014F00004EBC7E71E48103000880007010B1C48AA
:1015000014300088084370471948001D0188890677
:10151000FCD570471648001D018821F008010180A4
:1015200001880907FCD570470146114A0020121DA9
:1015300012880A4200D0012070470D49091D0A880F
:1015400082430A8070470A49091D0988C2B21140C6
:10155000074A1288024202D009B1012070470020D8
:1015600070470349091D0A8882430A8070470000BA
:1015700000280040F94910B5884202D10121C41465
:1015800086E0B0F1804F09D0F54988420DD10121A4
:101590000220FFF732FF0021022064E0012108460B
:1015A000FFF72BFF002101205DE0EE49884206D1C4
:1015B00001210420FFF721FF0021042053E0EA4924
:1015C000884206D101210820FFF717FF00210820DB
:1015D00049E0E649884206D101211020FFF70DFFBE
:1015E000002110203FE0E249884206D1012120205D
:1015F000FFF703FF0021202035E0DE49884202D1B9
:101600000121441444E0DC49884202D10121CC0488
:101610003EE0DA49884202D101210C0538E0D84980
:10162000884202D101214C0532E0D649884206D1D8
:1016300001214020FFF7E1FE0021402013E0D249C4
:10164000884206D101218020FFF7D7FE00218020AB
:1016500009E0CE4988420AD1841501212046FFF7CE
:10166000CCFE00212046BDE81040FFF7C6BEC849A9
:10167000884202D101210C040AE0C649884202D105
:1016800001214C0404E0C44988420AD101218C04A0
:101690002046FFF7A9FE2046BDE810400021FFF7D5
:1016A000A3BE10BD30B50288AC4BB24C98420DD0F1
:1016B000A0420BD0B0F1804F08D0A94DA84205D070
:1016C000A84DA84202D0A84DA84203D122F070052F
:1016D0004A882A43A54DA84206D0A54DA84203D06A
:1016E00022F44075CA882A4302808A8882850A8843
:1016F000028598420AD0A04208D0A54A904205D05F
:10170000A44A904202D0A44A904201D1097A0186AB
:101710000121818230BD30B5028C22F001020284A9
:10172000028C8388048B22F0020224F073050C885B
:101730002C430D8915434A882A43884DA8420BD073
:101740008C4DA84208D0924DA84205D0914DA84298
:1017500002D0914DA8420DD122F008054A8923F408
:1017600040732A4322F004058A882A438D891D4349
:10177000CB892B4383800483C9888186028430BD52
:1017800070B5028C22F010020284028C8488038BD4
:101790000D8823F4E6464FF6FF7303EA052535432B
:1017A0000E8922F0200203EA061616434A8803EA4D
:1017B00002123243694EB04202D06E4EB04215D191
:1017C00022F080064A8924F4406403EA021232437C
:1017D00022F040068A8803EA021232438E8903EA25
:1017E00086062643CC8903EA840434438480058337
:1017F000C9880187028470BD70B5028C22F48072A2
:101800000284028C8488838B0D8823F073031D432C
:1018100022F400730E894FF6FF7202EA06261E4379
:101820004B8802EA032333434C4EB04202D0514E60
:10183000B04215D123F400664B8924F4405402EAE7
:101840000323334323F480668B8802EA0323334364
:101850008E8902EA06162643CC8902EA0414344330
:1018600084808583C9888187038470BD70B5028CAC
:1018700022F480520284048C8288838B0D8823F4A6
:10188000E6464FF6FF7303EA0525354324F4005678
:101890000C8903EA043434434E8803EA06362643AF
:1018A0002E4CA04202D0334CA04205D122F48044F9
:1018B0008A8903EA8212224382808583C988A0F83C
:1018C0004010068470BD828B22F440628283828B3A
:1018D0004FF6FF7303EA01210A4382837047828B2C
:1018E00022F00C028283828B0A4382837047028B30
:1018F00022F440620283028B4FF6FF7303EA012158
:101900000A4302837047F0B5048C24F01004048469
:10191000078B048C4FF6FF7527F4734705EA0333F2
:101920003B4305EA02221A430C4B05EA0116984292
:101930000ED0104B98420BD0B0F1804F08D0084B1E
:10194000984205D0074B984202D0074B984225D1C8
:1019500024F02001314341F0100124E0002C01402B
:101960000004004000080040000C0040001000404F
:101970000014004000340140004C01400050014080
:101980000054014000180040001C004000200040AE
:1019900000400140004401400048014024F0A00301
:1019A0000B4343F0100102830184F0BD028B22F04F
:1019B0000C020283028B0A430283704770B5048CC9
:1019C00024F001040484058B048C4FF6FF7606EAAC
:1019D0000313134325F0F305F94A2B4390420ED02D
:1019E000F84A90420BD0B0F1804F08D0F64A9042AE
:1019F00005D0F64A904202D0F54A904202D124F036
:101A0000020201E024F00A020A4342F001010383CA
:101A1000018470BD2DE9F05F0D4604460888E84F4B
:101A2000DFF8A0C3DFF8A0834988AA882B894FF08C
:101A3000804960B3042832D04FF6FF7E082836D0A4
:101A4000208C9B4620F480502084A38B268C7046EB
:101A500000EA022223F473431A4300EA0B301043D6
:101A60000EEA013EBC420BD0644509D04C4507D07C
:101A7000444505D0D54A944202D0D54B9C4245D12D
:101A800026F4005141EA0E0141F4805143E0204622
:101A9000FFF794FFE9882046BDE8F05F86E720461F
:101AA000FFF731FFE9882046BDE8F05F1FE7208C93
:101AB00020F480702084B4F81CA0208C0EEA03135C
:101AC00013432AF0F30A0EEA012B43EA0A03BC424D
:101AD0000BD0644509D04C4507D0444505D0BB4ADE
:101AE000944202D0BA4A944204D120F4007040EAF1
:101AF0000B0002E020F42060084340F48070A383D0
:101B00002084E9882046BDE8F05FE8E626F402423A
:101B10000A4342F48051A08320462184E988BDE82D
:101B2000F05FD0E62DE9F0410C46002649880746D3
:101B3000012501B90226A288012A00D102252088A8
:101B400023890028384610D0FFF7DDFEE1883846AB
:101B5000FFF7CDFE23892A4631463846FFF72EFF90
:101B6000E1883846BDE8F04120E7FFF727FFE1882C
:101B70003846FFF71BFF23892A4631463846FFF7D0
:101B8000C2FEE1883846BDE8F041B0E610B50A88EB
:101B90004B88CC881A438B8823431A430B891A43FA
:101BA0004B8989891A430A43A0F8442010BD4FF697
:101BB000FF71818000210180C180418001727047E6
:101BC0000021018041808180C1800181418181812A
:101BD000C181704700210180418001228280C18043
:101BE000018170470021018041808180C180018195
:101BF0004181818170470029018802D041F00101B3
:101C000001E021F0010101807047002930F8441FF4
:101C100002D041F4004101E0C1F30E0101807047A0
:101C2000002A828901D00A4300E08A4382817047FA
:101C3000818270471143A0F848107047002A8289BA
:101C400001D00A4300E08A4382817047018921F074
:101C5000070101817047028922F070020A43028164
:101C6000704700B50346FFF7F6FF188940F00700FC
:101C7000188100BD70B516460D46602904464FF028
:101C8000010231460AD0FFF799FE29462046FFF7A8
:101C9000E2FF208940F00700208170BDFFF733FE8E
:101CA000F3E730B504894FF6FF7505EA03231343C4
:101CB000E4B20B432343038130BD10B50446FFF764
:101CC000F0FF208940F07700208110BD10B5044658
:101CD000FFF7E7FF208940F48040208110BD018597
:101CE00082827047028822F070020A4302807047A5
:101CF00070B50589048B068C25F007050D434FF65A
:101D0000FC410C4040F201110C434FF6FF7101EA17
:101D1000031126F022061143314305810483018417
:101D200070BD028B22F070020A4302837047028B5F
:101D30004FF6FF7322F4E04203EA012111430183CD
:101D40007047828B22F070020A4382837047828B35
:101D50004FF6FF7322F4E04203EA0121114381832D
:101D600070470029018802D041F0800101E021F094
:101D70008001018070470029818802D041F0040170
:101D800001E021F00401818070470029818802D0A0
:101D900041F0080101E021F008018180704700292D
:101DA000818802D041F0010101E021F00101818030
:101DB0007047028B22F008020A430283704700003A
:101DC000002C0140003401400004004000080040A5
:101DD000000C0040028B4FF6FF7322F4006203EA0E
:101DE000012111430183E9E7828B22F008020A43B3
:101DF0008283E3E7828B4FF6FF7322F4006203EAEB
:101E0000012111438183D9E7028B22F004020A43A6
:101E10000283D3E7028B4FF6FF7322F4806203EA5A
:101E2000012111430183C9E7828B22F004020A4396
:101E30008283C3E7828B4FF6FF7322F4806203EA4A
:101E4000012111438183B9E7028B22F080020A430A
:101E50000283B3E7028B4FF6FF73C2F30E0203EA6D
:101E6000012111430183A9E7828B22F080020A43FA
:101E70008283A3E7828B4FF6FF73C2F30E0203EA5D
:101E800001211143818399E7028C22F002020A4367
:101E9000028493E7028C22F008020A4302848DE751
:101EA000028C4FF6FF7322F0200203EA0111114366
:101EB000018483E7028C4FF6FF7322F0800203EA6D
:101EC00001111143018479E7028C4FF6FF7322F46C
:101ED000007203EA0121114301846FE7028C4FF67F
:101EE000FF7322F4006203EA01211143018465E7D4
:101EF000028C4FF6FF7322F4005203EA01311143C2
:101F000001845BE710B50123048C8B409C4304845F
:101F1000038C8A401343038410BD10B50423048C42
:101F20008B409C430484038C8A401343038410BD7C
:101F300030B50124058C00F118038C40A5430584BD
:101F400089B108290FD0091FC1F34E001844016858
:101F500021F4E041016001684FF6FF7303EA0222B9
:101F60001143016030BD03EB5100016821F07001A5
:101F700001600168F4E70029018802D041F0020104
:101F800001E021F00201018018E70029018802D058
:101F900041F0040101E021F0040101800EE7002975
:101FA000818802D041F0800101E021F08001818030
:101FB00004E7028822F00802028002880A430280B5
:101FC000FCE6828822F07002828082880A43828046
:101FD000F4E6028922F00702028102890A430281A3
:101FE000ECE6028922F08002028102890A43028122
:101FF000E4E68184E2E68185E0E68186DEE601872B
:10200000DCE68187DAE6A0F84010D7E6028822F401
:102010004072028002880A430280CFE6808ECDE6BD
:10202000008FCBE6808FC9E6B0F84000C6E6808C12
:10203000C4E6008DC2E602460020128A0A4200D0A1
:102040000120BBE6C9430182B8E602460020138A9C
:1020500092890B4202EA010202D0002A00D001203C
:10206000ACE6C9430182A9E6C64910B588420AD147
:1020700001218C032046FFF7B7F92046BDE8104048
:102080000021FFF7B1B9C049884202D101214C04B7
:1020900010E0BE49884202D101218C040AE0BC490B
:1020A000884202D10121CC0404E0BA4988420AD115
:1020B00001210C052046FFF7A0F92046BDE810409D
:1020C0000021FFF79AB910BD30B50446008A85B0EB
:1020D0000D464CF6FF710840E98801432182A18931
:1020E0004EF6F3100140A8882A8910436A890A43F2
:1020F0001043A081A08A4FF6FF410840A9890143FF
:10210000A1826846FFF714F99E48844201D10398E2
:1021100000E00298A1890904002900EBC00101EB4D
:102120000010296802DA4FEA410101E04FEA81011B
:10213000B0FBF1F06422B0FBF2F14FEA01114FEA7B
:1021400011136FF018056B4300EB8300A3891D0486
:102150004FF0320306D503EBC000B0FBF2F000F005
:10216000070005E003EB0010B0FBF2F000F00F00F9
:102170000843208105B030BD4FF4165101600021A5
:102180008180C18001810C2242818181704710B51C
:10219000038A4FF2FF0213400A884C8822438C883E
:1021A000C9880C4322431A43028210BD00210180DA
:1021B00041808180C18070470029818902D041F42B
:1021C000005101E021F400518181704710B5C1F345
:1021D000421301F01F040121A140012B07D0022B63
:1021E00007D01430002A026805D00A4304E00C30FE
:1021F000F8E71030F6E78A43026010BD002A828AB1
:1022000001D00A4300E08A4382827047028A22F0AA
:102210000F020282028A0A4302827047828922F4F4
:102220000062828182890A43828170470029818904
:1022300002D041F0020101E021F0020181817047EA
:10224000028A22F020020282028A0A430282704736
:102250000029018A02D041F4804101E021F480414B
:1022600001827047C1F30801818070478088C0F304
:1022700008007047818941F0010181817047028B1C
:10228000D2B20283028B42EA012101837047028BA2
:1022900002F47F420283028B0A43028370470029C3
:1022A000818A02D041F0200101E021F020018182E9
:1022B00070470029818A02D041F0100101E021F02D
:1022C0001001818270470029818A02D041F0080103
:1022D00001E021F00801818270470029818902D044
:1022E00041F4004101E0C1F30E01818170470029F2
:1022F000818A02D041F4006101E021F40061818211
:102300007047828A22F004028282828A0A43828291
:1023100070470029818A02D041F0020101E021F0DA
:102320000201818270470246002012880A4200D0D2
:1023300001207047C9430180704730B501F01F028A
:1023400001240025C1F3421304FA02F2012B0FD03D
:10235000022B0FD0838A4FEA11210088134204FA1E
:1023600001F400EA040001D000B10125284630BD87
:102370008389F0E7038AEEE70A0A01219140C94305
:102380000180704700380140004400400048004090
:10239000004C0040005000400CB500214C48019119
:1023A0000091026842F4803202604FF4A063026838
:1023B00002F400320092019A521C0192009A12B962
:1023C000019A9A42F3D10268920333D50121009118
:1023D00040490A6842F010020A600A6822F00302CB
:1023E0000A600A6842F002020A604168416041687E
:1023F0004160416841F480614160416821F47C1191
:102400004160416841F4E8114160016841F0807128
:10241000016001688901FCD5416821F00301416038
:10242000416841F0020141604168C1F38101022924
:10243000FAD10CBD00910CBD254810B5016841F0E2
:10244000010101604168244A114041600168234A4A
:1024500011400160016821F480210160416821F48C
:10246000FE0141604FF41F018160FFF795FF1C4999
:102470004FF00060086010BD154910B54868194A52
:1024800010F00C03184803D0042B01D0082B0BD0FC
:1024900002604968144AC1F30311121D515C0268BD
:1024A00022FA01F2026010BD4A684B6802F4701211
:1024B0004FF0020413F4803F04EB924202D04B68C9
:1024C0009B0301D5094B00E0064B5A43E0E70000AF
:1024D00000100240002002400000FFF8FFFFF6FE5F
:1024E00008ED00E000127A001400002000093D0011
:1024F00024490A20087000F01FFD02F030FA00F0B5
:1025000071FE00F0FAFD01F0DFFC01F02DFE00F09D
:1025100016FA02F04BFB012000F044FA194C012599
:10252000194E1A4FDFF86880DFF868B04EF6602A5F
:102530004FF00009A41C00BFC6F8A45102F055F9E1
:102540000FF07CFE01F0ECFF387808B100F0ADFE32
:10255000D8F80001002820880BD06428ECD3ABF811
:10256000A09000F08CFD002000F01CFAA4F8009070
:10257000E2E708B900F0C1FD20885045DCD8401CD6
:102580002080D9E72800002000802142FA000020A6
:10259000000021420010002042F6DF6305E01946EA
:1025A0000A00A1F1010189B2FAD10100A0F10100F4
:1025B00080B2F4D17047F0B5F349F44A01EB40031F
:1025C00003F5905103F58053C2E902130F88F04CD4
:1025D00000F5C06101F007061B88DFF8B8C3A55DF0
:1025E0000CEBD101BB421CD20B7800F560502B42A2
:1025F00000F007050CEBD00003D00178625D1143B9
:102600000DE0E54FBE5D33400B700178635D19420C
:1026100006D0D2680021118001787A5D11400170E6
:10262000F0BD087828430870F0BDD74970B501EBBC
:102630004002D64902F5905302F58052C1E90232B8
:1026400000F5C0621446D34B04F00706D24C03EBEE
:10265000D2021578A65D3540157000F5B0521546CA
:1026600003EBD20205F007051678655D00F56050B2
:102670002E40167003EBD00200F007001378205CA8
:10268000034013708A6800201080C968088070BDFC
:10269000F0B5BD4EBF4CBE4DBC4B002006EB40011B
:1026A00001F5905201F5805100F5B057BC46C3E9E1
:1026B000022104EBD7070CF0070C3F7815F80CC08B
:1026C00017EA0C0F11D00F88128897420DD200F52F
:1026D000C06204EBD20C02F007029CF800C0AA5CB6
:1026E0001CEA020F01D17F1C0F80401C80B2C82859
:1026F000D4D3F0BDF0B5A44EA64CA54DA34BC82035
:1027000006EB400101F5905201F5805100F5B057FC
:10271000BC46C3E9022104EBD7070CF0070C3F7855
:1027200015F80CC017EA0C0F11D00F8812889742C9
:102730000DD200F5C06204EBD20C02F007029CF847
:1027400000C0AA5C1CEA020F01D17F1C0F80401C54
:1027500080B2F628D4D3F0BDF0B58B4E8D4C8C4DA5
:102760008A4BF62006EB400101F5905201F58051AD
:1027700000F5B057BC46C3E9022104EBD7070CF0C3
:10278000070C3F7815F80CC017EA0C0F11D00F8812
:10279000128897420DD200F5C06204EBD20C02F011
:1027A00007029CF800C0AA5C1CEA020F01D17F1C42
:1027B0000F80401C80B2FA28D4D3F0BDF0B5724E21
:1027C000744C734D714BFA2006EB400101F59052A9
:1027D00001F5805100F5B057BC46C3E9022104EB76
:1027E000D7070CF0070C3F7815F80CC017EA0C0F50
:1027F00011D00F88128897420DD200F5C06204EB09
:10280000D20C02F007029CF800C0AA5C1CEA020F7E
:1028100001D17F1C0F80401C80B2FF28D4D9F0BDAD
:102820002DE9F0474FF0804000260682574DA888DA
:102830000A30A8802878401C287000F023FA2878F5
:10284000544C534F632808D92E7094F8E10139791C
:10285000084384F8E101FFF77FFF29784FF00A0968
:10286000B1FBF9F2A84609FB12104B4D072807D11E
:10287000FFF740FF94F8E101E978084084F8E101AE
:1028800098F80010B1FBF9F309FB1312022A05D1E5
:1028900094F8E121FB781A4384F8E121322907D129
:1028A000FFF7F6FE94F8E1012979084084F8E10188
:1028B00098F800005A280AD1FFF780FFB8F80210F4
:1028C0003648491CA8F8021006703548067098F87A
:1028D000000000F00F00022803D102F0CEF802F051
:1028E0006CF9B8F80210B1FBF9F309FB1312052AD1
:1028F00007D194F8E13195F805C003EA0C0384F898
:10290000E1312AB994F8E1217B791A4384F8E12175
:10291000B1F5967F07D059B1B1F5167F01D3A8F86C
:102920000260BDE8F08794F8E101A979084003E06E
:1029300094F8E101B979084384F8E101F1E73EB583
:1029400001210846FEF747FD48F6A040ADF8040017
:102950000120ADF800000020ADF80600ADF802003F
:102960004FF0804469462046FEF79CFE0121204638
:10297000FFF777FB012211462046FFF751F90121AD
:102980002046FFF738F93EBD00100020E00000208F
:10299000DE5F000800100020E65F00080C01002048
:1029A0000D0100202DE9F843054600214FF000609D
:1029B000FDF756FC4FF48060FDF720FC25208DF8D4
:1029C000000002268DF8016000248DF802408DF889
:1029D00003506846FDF717FC0E208DF800004FF0FD
:1029E00003088DF801808DF8026001268DF80360E0
:1029F0006846FDF708FC27208DF800008DF801607F
:102A00008DF802408DF803506846FDF7FCFB1D2051
:102A10008DF8000005208DF801008DF802408DF83A
:102A200003506846FDF7EFFB1E208DF800000427D9
:102A30008DF801708DF802408DF803506846FDF75F
:102A4000E2FB32208DF8000006208DF801008DF8A1
:102A500002408DF803506846FDF7D5FB2E208DF817
:102A600000008DF801408DF802608DF80360684623
:102A7000FDF7C9FB1C208DF800008DF801408DF892
:102A800002408DF803506846FDF7BDFB28208DF805
:102A900000008DF801708DF802408DF803506846F3
:102AA000FDF7B1FB17208DF800008DF801808DF83F
:102AB00002408DF803506846FDF7A5FBBDE8F8839A
:102AC0001CB50F210020FEF7F4FA4FF4805000905F
:102AD00000208DF804000C208DF8050001208DF8F1
:102AE00006006846FDF736FF4FF400600090684628
:102AF000FDF730FF1CBD1CB509210220FEF7D9FAF5
:102B00004FF40070009000208DF804000C208DF828
:102B1000050001208DF806006846FDF71BFF08211F
:102B20000220FEF7C6FA4FF4807000906846FDF769
:102B300011FF07210220FEF7BCFA802000906846B2
:102B4000FDF708FF06210220FEF7B3FA40200090AF
:102B50006846FDF7FFFE1CBD38B50120ADF800004A
:102B600004258DF8035002248DF802406946FD4883
:102B7000FEF7EBF92003ADF800008DF80350FA4D95
:102B80008DF8024069462846FEF7DFF94FF44070A1
:102B9000ADF8000014208DF803008DF8024069465E
:102BA000F248FEF7D2F94FF4E070ADF800001020C3
:102BB0008DF8030003208DF8020069462846FEF7D1
:102BC000C4F938BD38B50121E948FEF749FACE20ED
:102BD000ADF8000004248DF8034002258DF8025062
:102BE0006946E048FEF7B1F94FF20300ADF8000086
:102BF0008DF803408DF802506946DC48FEF7A5F9D0
:102C00003020ADF800008DF803408DF80250694681
:102C1000D548FEF79AF938BD38B50121D448FEF7FA
:102C20001FFA4FF41940ADF8000001248DF802405E
:102C300010258DF803506946CA48FEF786F9F8203A
:102C4000ADF800008DF802408DF803506946C74882
:102C5000FEF77BF94FF4F050ADF800008DF802401C
:102C60008DF803506946C048FEF76FF90420ADF8AF
:102C700000008DF802408DF803506946BD48FEF70C
:102C800064F938BDF0B5BC4CD4F80451BB48BD491B
:102C900000220378BA4890F880601DB10A7026F0CF
:102CA000010508E091F900509D4202DA6D1C0D709B
:102CB00003E046F0010580F88050D4F808512DB1AA
:102CC0004A7090F8805025F002050AE091F9015011
:102CD0009D4202DA6D1C4D7005E090F8805045F081
:102CE000020580F88050D4F80C512DB18A7090F80C
:102CF000805025F004050AE091F902509D4202DA65
:102D00006D1C8D7005E090F8805045F0040580F84A
:102D10008050D4F818512DB1CA7090F8805025F029
:102D200008050AE091F903509D4202DA6D1CCD704E
:102D300005E090F8805045F0080580F88050D4F800
:102D40001C412CB10A7190F8804024F010040AE074
:102D500091F904409C4202DA641C0C7105E090F881
:102D6000804044F0100480F88040874DD5F8104131
:102D70002CB14A7190F8804024F020040AE091F9C7
:102D800005409C4202DA641C4C7105E090F88040DA
:102D900044F0200480F88040D5F814412CB18A71A9
:102DA00090F8804024F040040AE091F906409C42EB
:102DB00002DA641C8C7105E090F8804044F0400415
:102DC00080F88040714CD4F800512DB1CA7190F850
:102DD000803023F080030AE091F907509D4202DA27
:102DE0006D1CCD7105E090F8803043F0800380F8D1
:102DF0008030D4F80471624DB5F8283E95F88160B2
:102E00001FB10A7226F0010508E091F908509D42B1
:102E100002DA6D1C0D7203E046F0010580F8815066
:102E2000D4F830512DB14A7290F8815025F0020546
:102E30000AE091F909509D4202DA6D1C4D7205E0DD
:102E400090F8815045F0020580F88150D4F8345153
:102E50002DB18A7290F8815025F004050AE091F9AD
:102E60000A509D4202DA6D1C8D7205E090F8815087
:102E700045F0040580F88150D4F838512DB1CA725C
:102E800090F8815025F008050AE091F90B509D4219
:102E900002DA6D1CCD7205E090F8815045F008050E
:102EA00080F88150D4F83C412CB10A7310F8811F8E
:102EB00021F010010AE091F90C209A4202DA521C2A
:102EC0000A73F0BD10F8811F41F010010170F0BDD0
:102ED0002B4B10B5A0332E49187800F001020A6080
:102EE0002C4AC0F340041460C0F38004D460C0F3E3
:102EF000C0041461C0F30014D461C0F340124A60EE
:102F0000C0F380128A60C009C8605878224A00F075
:102F10000101C2F888112149C0F340020A60C0F3E0
:102F200080024A60C0F3C0028A60C0F30012CA6027
:102F3000C0F34010086110BD10B501213C20FEF720
:102F400041FA01210846FEF73DFA144901201831E3
:102F50000860FFF761FEFFF7BBFFFFF733FEBDE838
:102F60001040F9E50008014000100140000C01404C
:102F7000000230000014014000002142F000002057
:102F800000100020AC0700200000224200802142F7
:102F9000A4012242A0012142008022428C812142D0
:102FA00010B50F48002404800E48D0F82411C0F852
:102FB000A44139B10C4800F61871B0F8180F00F1AF
:102FC00001000880084890F8F201800707D50448FE
:102FD000002201211038FEF723FE0448047010BDC2
:102FE000100400400000224200100020F1000020E8
:102FF00028B17649764B0A78DB791A430A7075490D
:10300000A1F87E0E70472DE9F04105460C281BD231
:10301000FDF71FFD704E06EBC520FDF755FD0024A2
:103020006E4FED024FF4806805EB4400304480B2EF
:1030300037F81410FDF70BFE641CA4B24445F3D31B
:10304000BDE8F041FDF711BDBDE8F08170B50C2879
:1030500014D20021C3026248604C4FF4806500BF67
:1030600003EB410292B2865C0244527806EB0222E4
:1030700024F81120491C89B2A942F1D370BD30B4A3
:10308000544A5649002041F2F41341F2B63400BFCD
:1030900032F8135021F81050401C5B1C9BB280B2D8
:1030A000A342F5D340F2645340F2965432F81350E1
:1030B00021F81050401C5B1C9BB280B2A342F5D398
:1030C00040F6640340F6960432F8135021F810508D
:1030D000401C5B1C9BB280B2A342F5D35FF020037F
:1030E00032F8134021F81040401C5B1C9BB280B2A8
:1030F000402BF5D330BC0A2085E730B500240A20E8
:10310000FFF7A4FF3548334941F2F41241F2B633D8
:1031100030F8145021F81250641C521C92B2A4B220
:103120009A42F5D340F2645240F2965330F814506C
:1031300021F81250641C521C92B2A4B29A42F5D3E8
:1031400040F6640240F6960330F8145021F812500D
:10315000641C521C92B2A4B29A42F5D35FF02002D2
:1031600030F8143021F81230641C521C92B2A4B210
:10317000402AF5D330BD17494FF480524FF43D53E8
:10318000002000BF21F81200521C92B29A42F9D3DB
:103190004FF4A0624FF4C06321F81200521C92B2A7
:1031A0009A42F9D34FF400624FF4106321F81200F1
:1031B000521C92B29A42F9D35FF0000221F8120039
:1031C000521C92B2802AF9D370470000E711002008
:1031D000DE5F00080010002000600008886E0020FC
:1031E0000060000830B5F9485221F94B8181F94A55
:1031F000002000BF33F8105000F5E064401C80B29E
:1032000022F814507E28F5D3F34B4FF6FF74F348A1
:103210005A5C194404EA022249780A43F0490280C0
:1032200009200870E949C82010310870487030BD85
:103230002DE9F0410546112822D2FDF70AFCE94E9E
:1032400006EBC520FDF740FC0024EF02E64D4FF4ED
:10325000806800BF05EB840235F82410927807EBF4
:103260004400304401EB022180B289B2FDF7EFFC4B
:10327000641CA4B24445EDD3BDE8F041FDF7F5BBB5
:10328000BDE8F08130B511280ED2D34CD64B0021C9
:103290004FF4006501EBC02292B2A25C23F811202A
:1032A000491C89B2A942F5D330BDC848017800292C
:1032B00009D00021017081714189CC488164416C41
:1032C00041F001014164704770B50024012805D028
:1032D000C74902282BD0032833D038E00020FFF75D
:1032E000D1FFC1490F204FF6FF72A1F8B800A1F835
:1032F000BA405E204FF4006321F81020401C80B2D9
:103300009842F9D3FDF7A5FBBA48FDF7DDFB002095
:10331000FFF78EFFB34D012405EBC420FDF7D4FB6E
:10332000641CA4B20A2CF7D3FDF79FFB0FE04FF407
:10333000005047F67E624454801C80B29042FAD31B
:1033400005E000204454801C80B2BE28FAD3AA496C
:10335000062048709D490120488170BD9B4A10B5E8
:1033600012890023C01C0321521E05E010F8014BF6
:10337000491C2344DBB289B29142F7DB184610BDE9
:10338000F0B5924904209D4C09899D4A9A4D891EA9
:103390000BE02718235C7F7805EB5006D35CD75DE4
:1033A000801C07EB0313337080B28842F1DBF0BD61
:1033B0009148C178807800EB01208449888170476A
:1033C0008D48C178007900EB01208049C8817047A1
:1033D000F8B57F49DFF8F4C1002231F81000009001
:1033E00085490220864B487010469CF80540143BE6
:1033F000EE4610E01EF8007001EB400603EB1715D7
:1034000007F00F072D78B570DF5D401C3D442A445E
:10341000F770D2B280B2A042ECD301EB400103249A
:10342000D21C8C70D2B203EB121402F00F0224787B
:10343000CC709A5C0A71042101EB4000ACF80A00E0
:10344000F8BDA0F58041B1F57A5F02D2A0F5005039
:1034500032E0A0F520717C2917D94031A0F5E07247
:10346000162901D890B27047A0F5C073162B01D869
:10347000E03821E0A0F500731F2B02D8A0F5A07062
:103480001AE0A0F5A0631F2B01D888B27047A0F501
:10349000F0711F2901D820380EE0BF2802D800F5AE
:1034A000807009E0A0F1C001BF2902D800F5886052
:1034B00002E01F2AEAD8203080B270474FF4C06281
:1034C000904202D200F5006034E0A0F5C061914264
:1034D00002D200F508502DE0A0F54061B72902D8CE
:1034E000A0F5E06026E0A0F59052A0F56061BF2A4B
:1034F00001D888B27047A0F5A053B3F57A7F01D206
:1035000098B27047A0F52053FF2B01D890B27047B6
:10351000A0F58052FF2A02D8A0F520600AE0FF291A
:1035200002D800F5807005E0A0F57061FF29EED8A3
:10353000A0F5807080B270472DE9F04302202E4E36
:10354000DFF8BC80002770703C46A8F114081F4DBE
:1035500023E0A889204480B2FFF773FFDFF8909042
:1035600006EB440C10F8091008EB111000788CF8E9
:103570000200A889204480B2FFF763FF10F8090019
:10358000641C00F00F01A4B218F801008CF80300CD
:103590009CF8021008443844C7B268798442D8D3F2
:1035A00006EB440003218170FF1CF9B208EB1113F4
:1035B00001F00F011B78C37018F80110017104208D
:1035C00000EB44006881BDE8F0830000F4000020B7
:1035D0007E3D01080010002000600008005000201F
:1035E000E011002000600008886E0020000002400A
:1035F00000100020006800088C7E002080800020E1
:10360000923F0108F0B5F84E0422F84DB178F078F9
:1036100002EB01210844A8810024F54F09E0A889A4
:10362000204480B2FFF70DFF3119641C4979C15560
:10363000A4B268798442F2D30620707001206881B8
:10364000F0BD30B5E84CE078A17800EB012080B205
:10365000FFF734FFE64901EBD005E078A17800EBF5
:10366000012080B2FFF72AFFE24900F00700085C62
:103670002978084328700620DC49607001204881C1
:1036800030BD30B5D84CE078A17800EB012080B295
:10369000FFF714FFD64901EBD005E078A17800EBE5
:1036A000012080B2FFF70AFFD34900F00700085C51
:1036B0002978084028700620CC4960700120488194
:1036C00030BDC948C178807801EB0020C74980B27D
:1036D0008881A0F56060023804D0C82800D02BE7AC
:1036E000652000E0012073E630B5C04CA089A0F54C
:1036F0006062233A15D00921BD4D012A17D0022A54
:103700001AD085F8E011FFF7D9FE05EBD005A089A6
:10371000FFF7D4FEB74900F00700085C297808439A
:103720002870B149062048700120608130BD85F8BD
:10373000E01100206070F4E70A2085F8E001F0E76E
:1037400030B5AA4CA089FFF7B9FEA94901EBD00515
:10375000A089FFF7B3FEA84900F00700085C2978AC
:103760000840A1492870062048700120608130BDC2
:103770002DE9F04FDFF870A2022100248AF8011031
:103780009AF804109AF8030001EB002080B2FFF7CA
:1037900058FEDFF858B241F290718842ABF80C0045
:1037A00003D0A0F5B852D03A54D18846404551D103
:1037B000924800252F4690F800C0A0F5A0591FE0C0
:1037C00009EB470141F204404E46085AFFF739FE23
:1037D000400806EB450336F8102023F808206D1C3E
:1037E000A0F5C062ADB26E2A08D806EB400006EB29
:1037F000450240886D1C22F80800ADB27F1CFFB264
:103800006745DDD37D48801C002690F800C01FE08E
:10381000B91909EB410141F20440085AFFF74EFE85
:10382000020900F00F0339F81220012000FA03F119
:10383000914305EB161209EB420215D002EB080189
:1038400006F00F030A88984082430A80761CF6B27D
:103850006645DDD30020BBF80C809BF80560684905
:103860005346DFF88C911CE0424406F00F031188A8
:10387000984001431180E9E708EB000703EB400C97
:1038800017F80950401C01EB151705F00F053F789C
:103890008CF802704D5D8CF803503D442C44E4B22A
:1038A00080B2B042E8D30AEB40030325E41C9D70CC
:1038B000E4B201EB141504F00F042D78DD70095DFE
:1038C0001971042101EB4000ABF80A00BDE8F08F4C
:1038D000F0B5454E454D00243079F178444F00EB6A
:1038E0000120A88109E0A889204480B2FFF7A9FD42
:1038F0003119641C8979C155A4B268798442F2D324
:103900000620707001206881F0BD2DE9F043364A31
:10391000364C02205070E0890023A0F5004085B2AB
:10392000E581184666793649DFF8D89016E000BF81
:1039300005EB000C19F80C8002EB400C01EB18179A
:1039400008F00F083F788CF8027011F80880401CCE
:1039500047443B448CF80380DBB280B2B042E7D3EB
:1039600002EB40020325DB1C9570DBB201EB131563
:1039700003F00F032D78D570C95C1171042101EBA0
:10398000400060811FE62DE9F047174E174CDFF825
:1039900060C03079F178012700EB012080B20A2164
:1039A000A0818CF8E0116770B0F5004F49D3164A3A
:1039B0000021A0F500401170A0810D4604F110080F
:1039C000DFF8489039E0A0894319DA0A88F8002026
:1039D00098F8010082421BD17019514203EBC122B9
:1039E000807929F8120026E08C7E0020F400002067
:1039F00000100020DE5F0008E65F000800240020C1
:103A00007E3F0108006000083B000020886E002017
:103A1000FFF70EFC98F80000FFF734FC98F8000060
:103A200088F80100A28971192A44404202EBC022A1
:103A3000897929F812106D1CADB260798542C2D324
:103A400011E0001DA08100250AE0A089284480B271
:103A5000FFF7F7FC71196D1C897900F80C10ADB2F5
:103A600060798542F1D3062070706781BDE8F087E8
:103A700070B505230A0ACCB2A0F50040F74980B220
:103A800045F6DB650E5CA64203D10E1876789642A9
:103A900005D0801C80B2A84201D8032BF2D800F5D3
:103AA000004080B270BD2DE9F041ED4CED4D6079E4
:103AB000A17900EB012081B2E889FFF7D9FFE88105
:103AC00002216170020AC3B23121E748A17000EB04
:103AD000121102F00F020978E170865C00EB1312FC
:103AE0002671127803F00F036271C35C31313144E7
:103AF00011441944C91CC9B2A371032700EB111268
:103B0000E771127801F00F012272405C60720920A7
:103B10006881BDE8F08130B50A280FD2D34CD44B70
:103B200000214FF4006500BF01EBC02292B2A25CFD
:103B300023F81120491C89B2A942F5D330BD2DE9E3
:103B4000F84FC84F05468946B97000F5004080B26D
:103B50000F21FFF78DFF4844A0F5004084B25B2D94
:103B60002BD9A5F15C0001040E0DB978A4F15C001D
:103B70004908C0F34E00C00801F00702CB08BA7034
:103B8000BC490EE00F1811F800C017F8017C07EBD4
:103B90000C2797403F0A00EB030C401E01F80C7005
:103BA00080B2B042EED10E180F5C16F8016C1844CA
:103BB00006EB07269640320A0A544FEAD42AE00A56
:103BC0000090B0EBD52F02D1C5F30A0600E0002625
:103BD000BAEBD42F03D1C4F30A077F1C01E04FF4E2
:103BE00000670098FFF74EFBE20AD2023046DFF88A
:103BF0007CB2DFF87CC27B1C0BE000BF02EB00084C
:103C0000A8EB090189B21BF801102CF81010401C18
:103C100080B29842F2D30098FFF70AFBB81B201A33
:103C200084B205EB0900A042C9D3BDE8F88F2DE9A5
:103C3000F0418B4F8B4D7879B979081A10F0FF015C
:103C400005D0E889A0F5004080B2FFF778FF8A49E7
:103C50000020844C0870642010344FF4004220701F
:103C60006070F978387902EB01210844A881B879AD
:103C700068710026DFF8F88120E0A8898219D10A4E
:103C800021706078814207D1B819C379484202EBAC
:103C9000C02128F811300FE0FFF7CAFA2078FFF7AB
:103CA000F1FA20786070AA89B9193244404202EBD7
:103CB000C022C97928F81210761CB6B268798642FB
:103CC000DBD32078FFF7B4FA0620787001206881F2
:103CD0001FE76448C8211030417001706049062018
:103CE0004870604901204881704710B55D4C103420
:103CF0006078FFF79DFAC82060702070FCF7B5FE71
:103D000057490620487057490120488110BD70B5B9
:103D1000544A10890B2805D158480379372B11D004
:103D2000382B0FD0FFF74CFB4D49887861284BD0DA
:103D300026DC11283FD01EDC98B3012838D010288B
:103D40002AD132E048498479143145790C5D4D5DC2
:103D500004EB0514C579007A4D5D085C2D0305EB75
:103D6000002020449081372B02D0BDE87040E7E46A
:103D7000BDE87040B8E4412823D060280CD126E08B
:103D8000772821D004DC622825D0632804D120E0E4
:103D9000872813D0D12823D01520487001205081C6
:103DA00070BDFFE7BDE87040E2E4BDE870408FE51C
:103DB000BDE87040A9E5BDE87040E4E5BDE87040AD
:103DC00093E7BDE870406EE6BDE8704081E70120F2
:103DD00002E0022000E00320BDE87040FFF774BA63
:103DE000BDE8704023E71F4810B51D49062304892C
:103DF00001224B70428110BD70B5FFF7C1FA1F4818
:103E0000174D184CC07837281BD006DC30280BD053
:103E100031280ED0342837D110E0382816D0422867
:103E200019D0452830D12BE028796071FFF749FC83
:103E30002AE028796071FFF7E5FB25E0FFF7D3FF63
:103E400022E0FFF7B5FAFFF7FCFB1DE0FFF7B0FA41
:103E5000FFF717FC18E0FFF748FF15E000600008C7
:103E60008C7E0020F40000207E3F010800500008F6
:103E7000886E002000D200203B00002080800020BF
:103E800068796071FFF743FF6189208901434FF032
:103E9000010002D115216970608100212181A0718A
:103EA0007EE71FB5694600900020ADF80400ADF82C
:103EB0000600ADF80800ADF80C000C20ADF80A00C3
:103EC0008F48FEF701F91FBD10B501218CB08803A2
:103ED000FDF778FA01210846FDF76BFA894C204678
:103EE000FCF746FC86480021001D009086480190A2
:103EF000102002908F20CDE903018020CDE905013B
:103F00008001CDE9081007910A9169462046FCF727
:103F10009CFC012202212046FCF7CCFC4FF4964089
:103F2000FFF7BFFF764C012240F225512046FEF7F5
:103F30004DF9012280212046FEF760F9012120463B
:103F4000FEF73AF96015ADF82C0003208DF82E002D
:103F500018206E4C8DF82F000BA92046FCF7F5FFBA
:103F60002015ADF82C0004208DF82F000BA9204659
:103F7000FCF7EBFF0CB010BD62484438416841F4D7
:103F800000514160416C4FF6FE721140416460493E
:103F90000120087070472DE9F0475948001D00883E
:103FA000DFF8709100F07F0000250126584C89F859
:103FB00000004FF00608A9F5FA77052804D002287A
:103FC00009D0208948B11BE0258187F801806681EE
:103FD000FFF76BF911E0268112E0207901281ED04D
:103FE00000281BD14FF41650FFF75BFF258187F89F
:103FF00001806681FFF759F92671208900280DD0CC
:104000002089CC46401C80B2208199F8001009F824
:104010000010B0F5C87F0ED96581258126E54FF4E3
:104020009640FFF73EFF258187F801806681FFF704
:104030003CF92571E1E70328F0D9604410F8020C3F
:104040000328EBD13348FFF789F9E07021890CEBA5
:10405000010212F8013C304A02EB10152D78AB42F8
:1040600009D100F00F001CF80110105C814202D150
:10407000BDE8F047C0E6152078706681BDE8F047DE
:10408000FFF713B970B51E4C40F22555294620465E
:10409000FEF753F9012805D129462046FEF76CF9B1
:1040A000FFF779FF08212046FEF73DF9012806D1E8
:1040B00008212046FEF73EF92046FEF7D7F840F2E9
:1040C000277529462046FEF738F9012808D12946E8
:1040D0002046FEF751F9002229462046FEF776F8E1
:1040E00040F2266529462046FEF727F9012805D12A
:1040F00029462046BDE87040FEF73EB950E6000074
:1041000000380140440002408D7E0020000801403C
:10411000F4000020808000207E3F010870B5FA4D39
:10412000FF22134605F5807606E000BF10F8014B2C
:1041300054402A5D5A40335D491EF7D243EA0220BB
:1041400070BD1FB5694600900020ADF80400ADF8C1
:104150000600ADF80800ADF80C000C20ADF80A0020
:10416000EA48FDF7B1FF1FBD38B501218804FDF70E
:1041700032F901210820FDF725F94FF40060ADF870
:1041800000000420E24C8DF8030069462046FCF74D
:10419000DCFE2015ADF8000003208DF80200182089
:1041A0008DF8030069462046FCF7CFFE4FF4964099
:1041B000FFF7C7FFD54C012240F225512046FEF7FC
:1041C00005F801212046FDF7F7FFD2490020A1F8AC
:1041D000040F0120A1F8F20E38BD2DE9F04FCE4EAC
:1041E000CE4C314696F801C0887891F803804A7920
:1041F0000B798146C74908EB0020002589B041F2C0
:104200006F7B4FF4FA5E01EB4001A6F16407BCF14D
:10421000050F70D018DC3346EA461B78BCF1010F5D
:104220006CD0BCF1020F68D0BCF1030F02D0BCF11E
:10423000040F5DD18DF8003051008DF801C081462A
:104240008DF802100020E5E0B34A4FF6FF79BCF18B
:10425000060F9378D27802EB0322AE4B03EB4202B7
:1042600002F500527DD0BCF10F0F41D0BCF1100F10
:104270003ED1DFF8A4C258459CF807309CF808C02E
:1042800004D809EA0328E044A2F80080704508D366
:10429000A1F58051138091F8601009EA0120604473
:1042A00010806570A5710020A179325C401C7A54A1
:1042B000491CC0B2A1710628F6D306219648FFF723
:1042C0002DFFA060A179C0F307227A54491CC9B21E
:1042D00001227854491CA17140F227718B48FDF7E7
:1042E00075FF00203554401CC0B20A28FAD9E57089
:1042F00009B0BDE8F08FE9E000E033E08DF8003070
:104300008DF801C08DF802908DF80380B1F8A000FF
:10431000010A8DF804108DF8050006215046FFF7BC
:10432000FDFE010AA0608DF806108DF8070065708B
:10433000A57100205246A179135C401C7B54491C96
:10434000C0B2A1710728F6D9012240F227716F4847
:10435000FDF73CFF00203554401CC0B20A28FAD9B2
:10436000C5E78AE08DF800308DF801C08DF8029025
:104370008DF80380B1F88000010A8DF804108DF8E3
:10438000050006215046FFF7C9FE010AA0608DF81E
:1043900006108DF807006570A57100205246A179BE
:1043A000135C401C7B54491CC0B2A1710728F6D98C
:1043B000012240F227715548FDF708FF00203554CF
:1043C000401CC0B20A28FAD991E700BF09EB0001EE
:1043D00059450DD84F4B0AEB400C03EB400303F556
:1043E00000531B884FEA13288CF803808CF80430A4
:1043F00071450DD3474B03EB4101A1F58051B1F855
:1044000060300AEB40014FEA132C81F803C00B71B6
:10441000401CC0B28242D9D89DF802105046C91C37
:10442000FFF77CFEA0609DF802300DF10301C0F3A0
:1044300007225A549DF8022001A9D44650546570B1
:10444000A5719DF802100020091D07E0A2791CF853
:104450000030BB54521C401CA271C0B28142F5D244
:10446000012240F227712948FDF7B0FE00203554A3
:10447000401CC0B20A28FAD939E727494FF6FF781D
:10448000584591F804C0497908EA0C2C614489B276
:1044900000D81180704500D311806570A57100208F
:1044A000A179325C401C7A54491CC0B2A171072822
:1044B000F6D9012240F227711448FDF787FE00204B
:1044C0003554401CC0B20A28FAD910E702EB032089
:1044D000A1F8A0006570A5710020A179325C401C94
:1044E0007A54491CC0B2A1710728F6D9012240F2C2
:1044F00027710648FDF76AFE00203554401CC0B203
:104500000A28FAD9F3E60000DF3F0108004800401E
:10451000000C014000100020D8820020080100207B
:1045200070B5624D2879002857D1287800260128D7
:1045300050D15F482E70B0F8040FE8BB5D4C5C4969
:104540002078B1F8F21E884244D1A87808280AD908
:1045500009212046FFF7E2FDA860A27AC1B291428C
:1045600010D1617A09E006215248FFF7D7FDA86013
:10457000E279C1B2914205D1A179B1EB102F01D1FD
:10458000FFF72BFE4A48B0F8040F012822D1484912
:104590002078B1F8F41E88421CD105214548FFF768
:1045A000BDFDA860A279C1B2914213D16179B1EB8E
:1045B000102F0FD1207900E00CE0E17800EB012012
:1045C0003D49A1F89C0000202654401CC0B20A2896
:1045D000FAD9AE70AE700120287170BD2DE9F0419E
:1045E000364D40F2255631462846FDF7A6FE2F4CA3
:1045F00008B331462846FDF7BFFE2079D8B12846DA
:10460000FDF734FE61792B4EC0B2012709B9307035
:10461000677127493078B1F8F21E88420BD12846DD
:10462000FDF724FE0146A0783154401CC0B2A070B2
:10463000072800D3277008212846FDF774FE0128BB
:1046400006D108212846FDF775FE2846FDF70EFE27
:1046500040F2277631462846FDF76FFE012815D136
:10466000144960786439095C401C60702846FDF785
:10467000F9FD6078A179884204D1002231462846AC
:10468000FDF7A4FD31462846FDF776FE40F226648C
:1046900021462846FDF751FE012805D1214628462E
:1046A000BDE8F041FDF768BEBDE8F08108010020DB
:1046B00000100020D8820020003000200048004078
:1046C00081070CD16421B0FBF1F201FB120141B969
:1046D0004FF4C871B0FBF1F201FB120008B10020E9
:1046E0007047012070472DE9F05F99460546DDE9E6
:1046F0000AAB0023A0F5FC6090460E46792802D351
:104700000120BDE8F09F4FF4FC64B04FDFF8C0C259
:1047100008E02046FFF7D4FF08B13B4400E06344C3
:10472000641CA4B2AC42F4D3761EF6B20024A94FA6
:10473000DFF8A4C20EE0385D40F2A321484303EB4A
:10474000C0132846FFF7BCFF10B1012C00D1634411
:10475000641CA4B2B442EED340F2A32108FB01F0E2
:104760009D4903EBC01049420844C9EB4912C2EB12
:10477000092100EB0110CAEB0A1100EB810000EBEC
:104780000B040120FCF7C8FCFCF7BEFE2046FCF73A
:1047900089FEFCF7B9FE0020B3E770B54FF4C8748A
:1047A000B0FBF4F303290DD2850706D14FF47A75D7
:1047B000B0FBF5F605FB160515B904FB13040CB99F
:1047C000521ED2B2024402EB90021A446423B0FBA0
:1047D000F3F0101A814A801E515C0844072190FBB7
:1047E000F1F201FB1200C0B270BD2DE9FC417C4822
:1047F0007C4990F8E121CB791A4214D07A487A4961
:1048000090F81A0E91F81C1ECDE90010764890F829
:104810001E3E90F8202E90F8221EB0F8240EFFF7CE
:1048200062FFBDE8FC8190F8E20189780842F8D087
:10483000FCF72FFE684F0546B0FBF7F367481E46AE
:10484000801E0188994238D003804FF4FC644FF4F5
:10485000B7784FF4B67C0FE02046FFF731FF38B150
:10486000434502D3A3F5B77304E0641CA4B205E08A
:10487000A3F26D13641CA4B26345EDD85A48DFF867
:1048800054C1A0F8244E00240EE05748B0F8220E80
:10489000FFF716FF08B1012C31D01CF80400984234
:1048A00004D81B1A641CA4B21C2BEED24E48641C04
:1048B0005B1CA0F8224EA0F8203E07FB16504FF4D8
:1048C0006162B0FBF2F1484B02FB1102A3F81E1E1D
:1048D0003C20B2FBF0F100FB1120A3F81C1E19468E
:1048E000A1F81A0E084690F8202E90F8221EB0F873
:1048F000240EFFF752FF3C49A1F8260E91E71D2B2D
:10490000D4D31D3BCEE710B501214FF0C050FCF7CA
:1049100062FD0120FCF700FCFBF760FE0120FCF7C4
:10492000EDFC4120FCF773FC0028FAD04FF48070B6
:10493000FCF7F5FC0120FCF7F7FCFCF7EBFDFCF7BE
:10494000E3FD01210846FCF78DFDFCF7DDFD47F690
:10495000FF70FCF7B4FDBDE81040FCF7D5BD10B505
:104960000420FBF764FE45F65A24A04206D0FFF768
:10497000CAFF21460420FBF753FE1AE001214FF045
:10498000C050FCF728FD002041F28831401C80B265
:104990008842FBD37B20FCF73AFC10B97A20FCF765
:1049A00036FCFCF73DFD01210846FCF75BFDFCF7FA
:1049B000ABFD0E480B4A4178927811430C4A417086
:1049C0000178D2791140017010BD00000085E2012C
:1049D0008033E101EE5F00088051010016010020E4
:1049E00000100020DE5F000800100020E111002010
:1049F000E65F000810B586B001210420FCF7E2FC58
:104A000001214807FCF7E7FC3020ADF81000002436
:104A10008DF8134004A92448FCF797FA3C20CDE90F
:104A200000040220039069460020FBF72FFE694630
:104A30001020FBF72BFE01210020FBF73FFE012198
:104A40001020FBF73BFE01210020FBF74BFE01216C
:104A50001020FBF747FE00210846FBF765FE00210A
:104A60000846FBF768FE01210020FBF73BFE012111
:104A70001020FBF737FE06B010BD0C4810B5B0F89B
:104A8000A01E0020FBF750FE0848B0F8A21E002030
:104A9000FBF751FE01210020FBF724FE0121BDE8B8
:104AA00010401020FBF71EBE00080140001000203F
:104AB00030B591B001214FF40470FCF783FC012163
:104AC0000846FCF776FC0F20ADF8400000248DF876
:104AD000434010A94748FCF738FA474D2846FBF7F2
:104AE00047FE464800904648CDE901044FF4C8709F
:104AF000CDE90304802005904000069080000790D7
:104B0000202008900002CDE9090469462846FBF7F9
:104B10009CFE01212846FBF7C2FE01208DF83000E3
:104B20008DF831000B944FF46020CDE90D04334C27
:104B300004208DF83C004C3C0BA92046FBF7D2FB2F
:104B4000072301220A212046FBF74CFC07230222FF
:104B50000B212046FBF746FC072303220C212046AD
:104B6000FBF740FC072304220D212046FBF73AFC0B
:104B700001212046FBF7E8FB01212046FBF7DAFB89
:104B80002046FBF7F4FB2046FBF7F6FB0028FAD1A2
:104B90002046FBF7F8FB2046FBF7FAFB0028FAD18A
:104BA00001212046FBF7FBFB11B030BD10B5FFF72C
:104BB0007FFFBDE81040FFF71DBFF0B50022104B8E
:104BC000104D1046642444F61C76002103EBC10707
:104BD00037F81070491CC9B23A446429F6D392FBE5
:104BE000F4F105EB4002401C91530022C0B20428AE
:104BF000EBD3F0BD00100140080002404C240140FE
:104C00003C8300200010002053EA020C00F0698071
:104C10002DE9F04B4FF00006002B1FBFB3FA83F5D0
:104C200003FA05F424FA05F65E4012BF1643B2FA01
:104C300082F502FA05F4C5F120051EBF22FA05FC33
:104C400044EA0C04203556EA044C4FEA144418BFD9
:104C5000641C4FF000084FF00009904271EB030C08
:104C600039D3002919BFB1FA81F701FA07F6B0FA72
:104C700080F700FA07F6C7F120071EBF20FA07FCED
:104C800046EA0C062037B6FBF4FCA7EB0507103FFD
:104C900007F01F0BCBF120060CFA0BFB2CFA06F6E3
:104CA00044BFB3460026202FA4BF5E464FF0000B42
:104CB0005BEA060C08BF4FF0010B19EB0B09ABFBCD
:104CC000027C48EB0608C01B06FB02CC0BFB03CCA6
:104CD00071EB0C01C1E70B46024641464846BDE870
:104CE000F08B13B54FF000004FF00001AFF30080E0
:104CF000BDE81C407047B2F120030AD5C2F1200381
:104D000001FA02F120FA03F300FA02F041EA03018A
:104D1000704700FA03F14FF000007047B2F1200332
:104D20000AD5C2F1200320FA02F001FA03F321FAB6
:104D300002F140EA0300704721FA03F04FF000014E
:104D4000704770477047704710B500F009F8006869
:104D500010BD10B5044600F003F8046010BD00005B
:104D6000004870475C860020004870475C86002041
:104D70007546FFF7F9FFAE4605006946534620F039
:104D80000700854618B020B5FBF726FABDE820409D
:104D90004FF000064FF000074FF000084FF0000BF7
:104DA00021F00701AC46ACE8C009ACE8C009ACE8AA
:104DB000C009ACE8C0098D4670470446AFF30080D7
:104DC0002046FBF7F4F9000001491820ABBEFEE7CE
:104DD000260002007047490050EAC12018BF042095
:104DE0004A0D18BF40F0010040F2FF72B2EB515F74
:104DF00008BF40F00200012808BF052070470000EE
:104E00002DE9FF4D21F0004807460C46B8F1795FC7
:104E100008DA00F0ADFF002801BF0020324904B0DD
:104E2000BDE8F08D3A4623461046194601F010F8C9
:104E3000054602462D480E460B460621784400F0F2
:104E40005DF82A46334601F003F8DDE90223824685
:104E50008B463846214600F0FBFF04460F4652467B
:104E60005B462846314600F0F3FF22463B460EF0F3
:104E7000C7FA07468A464FF0FF32284631460EF001
:104E800038FF1B4A90450ADA3A4653460EF0B8FA04
:104E900004B00022BDE8F04D134B01F089B8154A6B
:104EA0004245A8BFA8F500154FF00004B8BF124D49
:104EB00022462B460EF0A4FA0646884622462B468A
:104EC000002009490EF09CFA04460D463A46534626
:104ED000304641460EF094FA04B022462B46BDE817
:104EE000F04D01F065B800000000F03FA0F30000B5
:104EF0003333D33F0000E93F0000D23F2DE9F041BA
:104F00004F1E00EBC7010446D1E9000115461E46BD
:104F100037F006020DD02A46334600F099FF7F1E77
:104F200004EBC703D3E9002300F022FD37F00602AB
:104F3000F1D1022F25D0042F13D0062F18BFBDE8C2
:104F4000F0812A46334600F083FFD4E90A2300F0BB
:104F50000FFD2A46334600F07BFFD4E9082300F01A
:104F600007FD2A46334600F073FFD4E9062300F01C
:104F7000FFFC2A46334600F06BFFD4E9042300F01F
:104F8000F7FC2A46334600F063FFD4E9022300F021
:104F9000EFFC2A46334600F05BFFD4E90023BDE86E
:104FA000F04100F0E5BC0000024A002011070EF0BD
:104FB000A0BE000001FDFFFF02494FF000000EF00F
:104FC00066BE00BF0000F87F10F0004248BF4042BC
:104FD000B0FA80F310FA03F10AD0C3F11D0303F510
:104FE00080634FEA415002EB035202EBD12170473C
:104FF0004FF000007047FF2141EAD050C0057047D4
:10500000080000002DE9F74F144696B00021C4E9CE
:1050100002111799089121F00045CA498D4206DC1A
:105020001799C4E9000119B00020BDE8F08FC64906
:10503000DFF818A3A9423CDD0899C54E0029C54FE9
:10504000C54A1799534619DD0EF0DAF9554506D0D1
:10505000C24AC34B0EF0D4F9C4E900010AE04FF094
:10506000D352BF4B0EF0CCF932463B460EF0C8F996
:10507000C4E9000119B00120BDE8F08F00F078FC10
:10508000554506D0B54AB64B00F072FCC4E90001A4
:105090000AE04FF0D352B24B00F06AFC32463B4676
:1050A00000F066FCC4E9000119B04FF0FF30BDE824
:1050B000F08FAC49A942179978DB21F0004883466C
:1050C000A94AAA4B414600F0C3FE0022A84B00F0BB
:1050D0004FFC00F04DFE0990FFF776FF06460F46A5
:1050E0009D4A534600F0B4FE5A46434600F060FF26
:1050F00080468A46994A9A4B3046394600F0A8FEC7
:105100002A0D01250B924246534600F051FF032D14
:10511000C4E9000139D00B98C1F30A51401A05EBDC
:1051200045111139814230DA9248C346784400EB88
:105130000510CDF81CA00C90D0E90023304639466C
:1051400000F086FECDE9020102460B46584607995B
:105150000EF056F980468A4602460B465846079995
:105160000EF04EF9DDE902230EF04AF983460C9861
:1051700003913946D0E90223304600F069FE5A46D1
:10518000039B0EF03DF96D1CBDE708980028A2BFF7
:10519000099819B0BDE8F08F616881F00041616045
:1051A000099819B04042BDE8F08FFFE7C1F3130141
:1051B00041F480110E911799C1F30A51A1F2F53211
:1051C000511102F01F08C8F12002129200220C9225
:1051D0000D92694A7A4402EB810101F1140C0DA988
:1051E0005FF00607DCF80020DCF8045002FA08F350
:1051F000129AD1F800A025FA02F21A430E9BA2FBE4
:105200000356A2FB00329A4415449A4534BF4FF02E
:10521000010B4FF0000B51F8043C05EB0B0E7344EF
:10522000954234BF012200221644BBF1000F02D088
:10523000AB4202D903E0AB4201D2012200E00022DE
:105240003244C1F800A041E90223091FACF1040C6B
:105250007F1EC7D10898DDE90A6500F10050800F74
:1052600011900898099F8000FFF7AEFE80468A469D
:10527000384600F0DAFD6FF01D020EF03AFD0746E9
:105280003046059100F0D1FD6FF03D020EF031FD8A
:10529000CDE90310284600F0C8FD6FF05D020EF066
:1052A00028FD064602460B460191DDE9031000F099
:1052B0005FFB3A46059B00F05BFB4246534600F01D
:1052C00057FB00200D468346424653460EF098F8A1
:1052D0003A46059B0EF094F8DDE903320EF090F8A3
:1052E0003246019B00F064FEDFF89480234A434677
:1052F00000F0AEFD06460F46224A234B584629468B
:1053000000F0A6FD32463B4600F032FB0F46064653
:105310004FF0A84243465846294600F099FD3246D0
:105320003B4600F025FB179A12F0004F04D0119A6B
:1053300081F0004152421192C4E90001119819B064
:10534000BDE8F08FFB21E93F7CD90240FB21F93F0A
:105350007370032E8A19A33B000040543163621A14
:1053600061B4D03DFB21394183C8C96D305FE43F52
:105370000000E03FE0F0000068F00000182D445409
:10538000FB21F93D3326A611460B113C2DE9FF4DBB
:10539000054621F0004084B00C46B0F1795F0BDA8D
:1053A0002846FFF718FD042808BFFFF7FDFD284633
:1053B00008B02146BDE8F08D2A460B46104600F0A5
:1053C00047FD06460F462A46234600F041FD80462B
:1053D00026488A4632463B4605217844FFF78EFD33
:1053E00083461098029160B3214A224B40465146B1
:1053F00000F02EFDCDE900015A4640465146029B81
:1054000000F026FD82468846DDE906014FF0FF32B6
:105410000EF06FFC524643460DF0F2FF32463B461B
:1054200000F016FDDDE906230DF0EAFFDDE90023BB
:105430000DF0E6FF08B02A462346BDE8F04D00F027
:10544000B7BD0B465A463046394600F001FD084AC2
:10545000084B00F08DFA4246534600F0F9FC08B0C4
:105460002A462346BDE8F04D00F082BAFAEE00006D
:10547000495555555555C5BF2DE9F04D044688B0E1
:105480008F4821F00047164698460D460691874200
:1054900006DA2046294600F06BFC002800F0AC80BC
:1054A0008848B8421CDC06980028BCBF85F000453F
:1054B00088F00048844A854B2046294600F078FD54
:1054C00004460D4632464346814882490DF098FF16
:1054D00022462B4600F04CFA002604460D46B04604
:1054E00022462B461046194600F0B2FC8B468246F7
:1054F00002460B4600F0ACFCCDE9020102467648BC
:105500000B4606217844FFF7F9FCCDE9000173480A
:1055100006217844DDE90223FFF7F0FC52465B46A2
:1055200000F096FCCDE9020152465B462046294632
:1055300000F08EFCCDE904019DE80F0000F018FAA0
:10554000DDE9042300F084FC3246434600F010FA03
:1055500052465B4600F07CFC3246434600F008FAB7
:1055600080460E46DDE904015D4A5E4B00F070FCAA
:105570004246334600F0FCF982468B4622462B46D3
:1055800000F0F6F980464F480E46B84210985BDCB2
:10559000FFF71AFD074642463346029100F0E8F94C
:1055A000CDE90001424633461046194600F050FC52
:1055B000DDE9002300F084FA52465B460DF020FF3F
:1055C00022462B4600F0F4FC01220EF092FB3A46F4
:1055D000029B00F0EDFC04460D460698022101EA0C
:1055E000A070C0F10100FFF7EFFC08B022462B4687
:1055F000BDE8F04D00F02CBC1098401C384320430F
:105600000BD01098012812D008B022462B46BDE8D6
:10561000F04D0020344900F053BA08B025F00043A3
:105620002246BDE8F04D0020304900F049BA20463E
:105630002946FFF7D0FB042808BFFFF7B5FC20463A
:1056400008B02946BDE8F08D012802BF404608B0E9
:10565000BDE8F08D00270B463A462046294600F06B
:10566000A7FC52465B4600F0A3FC04460D464246AA
:10567000334600201C4900F023FA83463A46884608
:105680003346104600F0E4FB0022184B00F070F99E
:1056900006468A4622462B463846414600F0D8FB4D
:1056A0003246534600F064F95A46434600F0D0FBB8
:1056B00008B03A464346BDE8F04D00F059B9000045
:1056C0000000303E2894E53F182D4454FB21E93F6B
:1056D000075C143326A6813CF8ED00001AEE0000AA
:1056E000635555555555D53F0000F0BF0000F03FBC
:1056F00000B5284B21F0004287B09A42DCBF00225F
:10570000134631DD244B9A420DD168B94FF00100A8
:10571000FFF71FFB002207B01346104611465DF845
:1057200004EB00F0CDB906DB07B04FF001025DF8E5
:1057300004EB0EF0DEBA02AAFFF764FC10F00301DE
:1057400004BF0DF1080CBCE80F000DD001200129A9
:105750000ED0022914D00DF1080C0090BCE80F0007
:10576000FFF714FE07B000BDFFF74AFB07B000BD0E
:105770000DF1080C0090BCE80F00FFF707FE05E0F4
:105780000DF1080CBCE80F00FFF73AFB07B081F001
:10579000004100BDFB21E93F0000F07F00B5294B2F
:1057A00021F0004287B09A4203DC002213460092A7
:1057B00033E0254B9A420DD168B94FF00100FFF755
:1057C000C8FA002207B01346104611465DF804EBF4
:1057D00000F076B906DB07B04FF001025DF804EB8C
:1057E0000EF087BA02AAFFF70DFC10F003014FF08C
:1057F00001000DD0012914D002291AD00DF1080C96
:10580000BCE80F00FFF7FCFA07B081F0004100BDD3
:105810000DF1080C0090BCE80F00FFF7B7FD07B0D2
:1058200000BD0DF1080CBCE80F00FFF7E9FA07B066
:1058300000BD0DF1080C0090BCE80F00FFF7A6FDBD
:10584000E2E70000FB21E93F0000F07F2DE9F04195
:1058500006460F460DF0EEFC04000D4618BF012071
:10586000284320F00040C0F17F6000F1E040C00F0D
:105870000ED0301C18BF0120384320F00040C0F18A
:105880007F6000F1E040C00F04BF0120FFF761FA24
:1058900020462946BDE8F08110B51A4B21F00042A0
:1058A000012486B09A4203DC00221346009424E0CF
:1058B000154B9A420DD168B94FF00100FFF749FA34
:1058C000002206B01346BDE810401046114600F015
:1058D000F7B806DB06B04FF00102BDE810400EF04D
:1058E00008BA02AAFFF78EFB00F00100A4EB40000B
:1058F0000DF1080C0090BCE80F00FFF7BDFD06B0ED
:1059000010BD0000FB21E93F0000F07F21F00042C4
:10591000A2F16052B2F5801F01F0004328BFD2F11E
:105920007F6C0BD95FEA001C43EAC20242EB507065
:1059300018BF704728BF20F001007047B2F5801FE4
:10594000BCBF184670474FEA410C1CF5001F02D23D
:105950000846FFF750BB70B50DF01EFC0000008933
:10596000FFF7F6BF4FF00040A0F580007047000041
:1059700010B591EA030F48BF83F000430DF148854D
:10598000841A71EB030C05D2121943EB0C03001BB4
:1059900061EB0C01DFF824E14FEA1154A4EB135C36
:1059A0001EEA430F18BF9EEA445F73D023EA0E033A
:1059B000DCF1200E21EA045143F4801332D322FAA1
:1059C0000CFE10EB0E0023FA0CFE41EB0E01CCF1A5
:1059D000200E03FA0EFE10EB0E0051F10001B1F59E
:1059E000801FCCF1200E32D201EB045112FA0EF2DC
:1059F000BDE8104058BF7047401C38BF5FEA420204
:105A000018BF7047002814BF20F0010041F10001C9
:105A10004FEA410313F5001F38BF7047A1F1C041A1
:105A200000F0C0BA012A43EB0302ACF1200CDCF118
:105A30001F0E32BF4FF0000E23FA0CF310EB0300E1
:105A400041EB0451B4EB115FD0D0A1EB045101F54F
:105A5000801149085FEA300001EB04510ED350F188
:105A6000000038BF12FA0EFE08D1BDE81040C9E7A9
:105A7000401C38BF5FEA4202CAD1C3E7BDE810400C
:105A80004FEA410313F5001F38BF7047A1F1C04131
:105A900000F088BA9EEA445F08D011EA5E0FBDE8C4
:105AA000104004BF01F0004100207047BDE81040E5
:105AB00070B50DF071FB00BF64FBBE3E0000E0FF5F
:105AC0002DE9C04130B4DFF8A0C23CEA111418BF80
:105AD0003CEA131400F0EC8081EA03051CEA11147F
:105AE00044EAD57418BF1CEA131500F0C780A4EB74
:105AF00005044FF0004545EAC12145EAC32341EAC8
:105B0000505143EA525304F17F74994204F5003432
:105B10004FEAC0204FEAC22208BF904200F09C80AA
:105B20004FEA13650FF24016765D4FEA134506FB08
:105B300005F7C7F1807706FB07F74FEAD737A7FBD2
:105B400003687642C8F58038A7FB06CE38BFA8F1B7
:105B5000010807FB08E64FF0000EA6FB028CE6FBEF
:105B600003CEDCF1000CCEF1004E38BFAEF1010ED9
:105B7000A6FB0C584FF000074FF00005E6FB0E8720
:105B8000A1FB08C6A0FB07CE16EB0E0645F10005EB
:105B9000E1FB076515F1E04E7EBFA4F580345FEAB6
:105BA00046066D4116F1800745F100054FEA1727BB
:105BB0004FEA066647EA0567A6F1DE46B6F1805F62
:105BC0004FEA15251FD9384624F0010C05EBC471A6
:105BD000BCF1FE6F01EB0C1102D8F0BCBDE80081F6
:105BE00024425CBF01F5801E9EEAC47F02D4F0BC53
:105BF000BDE80081244238D4F0BCA1F1C041BDE829
:105C0000004100F0CFB94FEAD22242EA43524FEAB4
:105C1000D323A7FB02864FEAD02040EA415007FB7E
:105C200003661EEA0E0F4FEAD12105FB026658BF3C
:105C3000A6EB0056B6EB00564FEA520E4EEAC37E74
:105C400018EB0E0E56EB530EBDD518EB02085E4155
:105C50007F1C55F10005B6E74FF480154FF00007A3
:105C60004FF000064FF00008ADE7F0BC4FF0000029
:105C700001F1C04101F00041BDE8008111EA0C1FB3
:105C80000CEA131500D00CE013EA0C1F00F025807D
:105C90004FF00000F0BC81EA030101F00041BDE8D3
:105CA0000081F0BCBDE8004181EA030100F07AB94F
:105CB000F0BCBDE8004170B50DF06EFA097EFC3E07
:105CC00000F007B881EA03014FF0000001F0004145
:105CD000704781EA030100F065B9F0BCBDE80041FE
:105CE0004FF0000021497047FFFDFBF9F7F5F4F292
:105CF000F0EEEDEBE9E8E6E4E3E1E0DEDDDBDAD867
:105D0000D7D5D4D3D1D0CFCDCCCBCAC8C7C6C5C4C4
:105D1000C2C1C0BFBEBDBCBBBAB9B8B7B6B5B4B3DB
:105D2000B2B1B0AFAEADACABAAA9A8A8A7A6A5A4C6
:105D3000A3A3A2A1A09F9F9E9D9C9C9B9A9999988A
:105D40009797969595949393929191908F8F8E8E2D
:105D50008D8C8C8B8B8A89898888878786858584BA
:105D600084838382828181800000FF070000F87FA6
:105D70004FEA41034FEA5353A3F58063D3F11E0367
:105D8000C8BFD3F1210C0CDD4FF0004242EAC12222
:105D900042EA505232FA03FC8CEAE17CACEBE1704F
:105DA0007047102BC4BF0020704703F5787CBCF10E
:105DB000FF3F04D06FF0004282EA2100704770B5C7
:105DC0000DF0EAF94992248000207047F2E70000C4
:105DD0004FEA1153A3F58063D3F11E03A8BFD3F19B
:105DE000200C08DB4FF0004242EAC12252EA505236
:105DF00032FA03F0704709420BD4102BC4BF0020C5
:105E0000704703F5787CBCF1FF3F05D04FF0FF30C1
:105E100070474FF00000704770B50DF0BDF900BF3E
:105E20004992248000207047F0E7B0FA80F310FA1E
:105E300003F10AD0C3F11D0303F580634FEA41501B
:105E40004FEA035202EBD12170474FF00000704738
:105E5000DFF848C170B51CEA111E1EBF1CEA1315FD
:105E60009EEA0C0F95EA0C0F00F06F8081EA0304A4
:105E700023EA4C134EEAD47E21EA4C1141F48011FE
:105E800043F48013AE44A1FB024CA0FB0365AEF1CA
:105E90007F7E361955EB0C05A1FB034C4CF100033A
:105EA000A0FB021C16EB0C06654153F100030942EE
:105EB00018BF46F0010613F4007F0BD14FEA0331FF
:105EC0004FEA0530340341EA155140EA16506FF0AD
:105ED00003020AE04FEAC3214FEAC520F40241EA77
:105EE000555140EA56506FF0020202EB2E4201EB90
:105EF000025585EACE710AD05FEA440C18BF24F03F
:105F0000004450F1000041F1000120EAD47040F259
:105F1000FE7C624500D270BDA84214BF4FF08044A1
:105F20004FF04044002E08BF0024BEF1806FA8BF90
:105F3000A1F1C041BDE8704080F234804FF0000014
:105F400001F1C04101F0004170479EEA0C0F0CEADC
:105F5000131518BF95EA0C0F06D04FF0000081EA28
:105F6000030E0EF0004170BD0DF016F98900013EE0
:105F700000F007B800F009B84FEA430C5FEA5C5C38
:105F800008D081EA030100F00DB84FEA410C5FEA46
:105F90005C5CF6D14FF00000014970470000FF073C
:105FA0000000F87F0808A0F500114FEA31017047A2
:105FB00091EA030F10B581F000413FF5E1AC83F0A9
:105FC00000430DF025BA401058BFC0F140404910C1
:105FD00058BFC1F140418142EFF300807047010298
:105FE000040810204080FEFDFBF7EFDFBF7F1F1C81
:105FF0001F1E1F1E1F1F1E1F1E1F0000000000006F
:106000001000D8BA000000002020202020202020EE
:106010002020202020202020202020202020202080
:106020002020202020202020202020202020202070
:10603000F409FF0BF401E703640EC70EDC0EFF0E3C
:106040009001FE03000000000000000000000000BE
:106050008300000000000000000000000F00FFFFB0
:10606000FFFFFFFFFFFFFFFFFFFFFFFFFFFFFFFF40
:10607000FFFFFFFFFF000000000000000000000025
:106080000000000000000000000000000000000010
:106090000000000000000000000000000000000000
:1060A00000000000000000000000000000000000F0
:1060B00000000000000000000000000000000000E0
:10E4D00030B50024012512E00B185B1E5B089A4240
:10E4E00006D81DB9091A491C04EB51041946F1E775
:10E4F0001DB1081A401C04EB5004581C002588422A
:10E50000EAD3204630BD70B50025012310E00C1A77
:10E51000641C05EB5404A24201D2012600E000264F
:10E520009E4208D003B125460844401C4008002301
:10E530008842ECD370BD03B925460144491E490801
:10E54000E3E70346012101E05B084900002BFBD112
:10E5500019B1491E02460020BAE74FF0FF3070475C
:10E560000346012101E05B084900002BFBD119B1F2
:10E57000491E02460020C6E74FF0FF30704770B5D5
:10E58000F64CF74DA06D2844C0F34F0004F007F897
:10E5900000286079F3494FEAC07001D0A8B126E0A5
:10E5A000002811D0A06D42195010C31700EB537012
:10E5B00001EBE00120F00700C0EB6200EA4A0B78B3
:10E5C000805C03430B70012070BDA06D4219501098
:10E5D000C31700EB537001EBE00120F00700C0EB24
:10E5E0006200E14A0B780832805C03400B70002027
:10E5F00070BDDE4A0020A2F8180E1046B0F8880E52
:10E6000060B91046A0F8861ED448D549C06D491E91
:10E6100008441146C0F34F00A1F8880ED348D349EF
:10E62000B0F8880EA1F88A0E704770B5D04BCB4970
:10E6300003EBD00200F007050846CB4C4079127876
:10E640004006655D0E7B000E2A40012E487101D008
:10E650005AB970BD002AFCD00A8C03EBD20302F039
:10E6600007021B78A25C1342F3D040F0010048710E
:10E6700070BD70B5BE4BB94903EBD00200F0070581
:10E680000846B94C407912784006655D0E7B000E55
:10E690002A40012E487102D0002A0ED10AE0002A39
:10E6A0000BD10A8C03EBD20302F007021B78A25CA9
:10E6B000134202D040F00100487170BDAC4901EB3B
:10E6C000D00100F007000A78A749085C0242A3487D
:10E6D000417904D0CA0702D041F0010101E001F004
:10E6E000FE0141717047A24901EBD00100F0070023
:10E6F0000A789D49085C02429848417904D1CA07CA
:10E7000002D041F0010101E001F0FE0141717047CA
:10E71000974901EBD00100F007000A789249085CA4
:10E7200002408E48417901F001031A4302D041F0C2
:10E73000010101E001F0FE01417170478C4901EBDC
:10E74000D00100F007000A788749085C024083483E
:10E75000417901F001035B1E1A4203D001F0FE0172
:10E760004171704741F00101FAE7F0B5DFF8ECE1E3
:10E770007D4D71469EF80D604C797D4908357A4B88
:10E7800000F0070201EBD001012E2ED19EF80C60A3
:10E79000012E04D00A2828D2E00728D1F0BD6F4E00
:10E7A000DFF8CCC10A28378C07F007060CEBD70737
:10E7B00006D2E007F2D03878AC5D2040387016E021
:10E7C0003F789E5D3742E9D0E40714D00C789A5C1C
:10E7D00014430C70674A9EF80E1022F81100491C71
:10E7E0008EF80E10F0BD0870F0BDE00703D0087879
:10E7F0009A5C1043F7E70878AA5C1040F3E72DE92C
:10E80000F04756494A79D2070ED00D7B584ADFF8B7
:10E81000589100F0070402EBD003012D06D01878C0
:10E8200019F8041008431870BDE8F0874E4D002019
:10E830008E7B0835DFF83CA110E000BF3AF810C02D
:10E84000401C02EBDC070CF0070C97F8008015F871
:10E850000CC0C0B208EA0C0887F80080B042EDD9BD
:10E86000088C02EBD00200F007001678285C064006
:10E870001670187819F80420104318700020887357
:10E88000D2E710B535490122394B4A730A7308841F
:10E890004A7903EBD0035206120E334C4A7100F052
:10E8A00007001B78205C034202D042F0010048714F
:10E8B00010BD70B42949F83808284A798D7902F0DA
:10E8C000FE0605F0010346EA030420D2DFE800F06B
:10E8D00004091014161A1F0E42F0FE0000EA52003E
:10E8E00003E002F0010040EA5200487170BC70473A
:10E8F00065F35F028A71F9E74C71F7E74C716808BC
:10E900008871F3E70120904306434E71EEE770BC37
:10E9100002214FF474606CE62DE9F0410F4C124F68
:10E920000F4E60790F4DC107204607F10807806D33
:10E9300030443CD0C0F34F0003F031FE0C4A6FF47A
:10E94000D051C8B1A06D008801EAD001114400F097
:10E9500007000A78385C02400A7036E03000002078
:10E96000A49FFFF7CD070020DE5F00080010002005
:10E9700000100020AC050020A36D1E447010C717C6
:10E9800000EB577005EBE00520F00700C0EB6606D2
:10E99000F6482F78365C37432F701B8801EAD30185
:10E9A000114403F007030A78C05C0243D4E7411026
:10E9B000CA1701EB527105EBE10221F00701C1EB2F
:10E9C00060001378C05D03401370A06D801CA065CB
:10E9D000BDE8F0812DE9F041E54CE74DE54E607969
:10E9E000E24FC1072046806D2844C0F34F0013D08A
:10E9F00003F0D5FDC0BBA06D41194810C21700EB54
:10EA0000527006EBE00220F00700C0EB61001378C3
:10EA1000C05D0343137032E003F0C1FDD34BD74A0E
:10EA200008330028A06D6FF4D0511ED005444FEA82
:10EA3000650C4FEAEC7E0CEB5E7C06EBEC062CF0F2
:10EA4000070CCCEB650596F800E0EB5C0EEA030ED4
:10EA500086F800E0008801EAD001114400F00700C8
:10EA60000A78385C024309E009E0008801EAD00135
:10EA7000114400F007000A78185C02400A70A06D8B
:10EA8000801CA065A4E72DE9F041DFF8E4E20F4621
:10EA90000021DEF8603043EA0222BEF810301A444A
:10EAA0004FF6FC7302F01F0403EAD205CEF8602093
:10EAB000A0F182020F2A59D2DFE802F0085811585B
:10EAC0001C5826582F58385842584C0007F00F0051
:10EAD0002246F6F710F907468C460F2006E0F8B2FA
:10EAE0002246F6F708F907468C46FF20A040C043AF
:10EAF000C61740E0C7F30B002246F6F7FCF80746BE
:10EB00008C4640F6FF70F1E7B8B22246F6F7F3F80C
:10EB100007468C464FF6FF70E8E7C7F3130022461E
:10EB2000F6F7E9F807468C469548DFE727F07F407F
:10EB30002246F6F7E0F807468C466FF07F40D5E7AF
:10EB400027F070402246F6F7D6F807468C466FF05D
:10EB50007040CBE738460E462246F6F7CCF807461B
:10EB60004FF0FF30A0408C46C04304E0DEF8581060
:10EB7000891DCEF8581081496B18D3E90021314026
:10EB800002403A4341EA0C01C3E9002120E77849F9
:10EB900010B50A6E4FF6FC7342EA00200A8A104450
:10EBA00000F01F0208664A8203EAD0008882734997
:10EBB0000144D1E90001F6F7B1F810BD30B56C4958
:10EBC0008A6D32F8024B250A803D092D15D2DFE807
:10EBD00005F005140B1416141C14220000EB04207D
:10EBE00080B24FF4E06304E000EB042080B24FF405
:10EBF000006303EB5000C8828A65C88A30BD00EB11
:10EC0000042080B24FF4A063F3E700EB042080B24D
:10EC10004FF48053EDE700EB042080B241F2E8337B
:10EC2000E7E710B5524CA16D31F8020B020A842AB5
:10EC300002D0862A11D10AE0C0B2607011F8022B0E
:10EC400040EA022020830020A165207005E0C0B2C8
:10EC50006070A165FFF7B2FF2083208B10BD70B5F7
:10EC6000434C4FF6FF75A06D30F8023BA06502885B
:10EC700003F47F41DBB205EA0225236641EA122153
:10EC80002B43A1F50645803D01D13E490CE0A1F59D
:10EC90000645823D03D103F12023A36262E0A1F582
:10ECA0000645843D03D138491944A1625AE0A1F5D3
:10ECB0000645863D01D13549F6E7A1F50645883D73
:10ECC00001D13349F0E70025A1F50440823805D190
:10ECD000D0B2FFF75CFF00F00F0040E0A1F5044068
:10ECE000843804D1D0B2FFF752FFC0B237E0A1F5AB
:10ECF0000440863805D1D0B2FFF749FFC0F30B00BE
:10ED00002DE0A1F50440883804D1D0B2FFF73FFFD1
:10ED100080B224E0A1F504408A3805D1D0B2FFF7D3
:10ED200036FFC0F313001AE0A1F504408C3805D17A
:10ED3000D0B2FFF72CFF20F07F4010E0A1F5044097
:10ED40008E3805D1D0B2FFF722FF20F0704006E0E8
:10ED5000A1F50440903807D1D0B2FFF718FFA062A8
:10ED60002570A06D801CA065A06A70BDDE5F0008E4
:10ED700030000020CD070020A49FFFF700100020E6
:10ED8000FFFF0F00001E0020001A002000300020AE
:10ED9000D0370020800B07D0012809D002280BD0E3
:10EDA00003280DD000207047F748B0F83A0E70479E
:10EDB000F548B0F86E0F7047F348B0F8720F70471F
:10EDC000F148B0F8760F7047800B07D0012809D0C2
:10EDD00002280BD003280DD000207047EA48B0F875
:10EDE0007A0F7047E848B0F87E0F7047E648B0F8F1
:10EDF000820F7047E448B0F8860F7047800B07D049
:10EE0000012809D002280BD003280DD0002070471C
:10EE1000DD48B0F8380E7047DB48B0F86C0F70472B
:10EE2000D948B0F8700F7047D748B0F8740F7047E2
:10EE3000800B07D0012809D002280BD003280DD061
:10EE400000207047D048B0F8780F7047CE48B0F82F
:10EE50007C0F7047CC48B0F8800F7047CA48B0F8B4
:10EE6000840F7047800B07D001280CD0022811D0E6
:10EE7000032815D000207047C348C349B0F8380EA6
:10EE8000B1F83A1E12E0C048BF49B0F86C0FB1F8B3
:10EE90006E1F0BE0BC48B0F8700F00EB00407047ED
:10EEA000B948B949B0F8740FB1F8721F00EB0140CE
:10EEB0007047800B0AD001280FD0B3490228B1F85F
:10EEC000821F11D0032813D000207047AE48AE49EE
:10EED000B0F8780F91F87A1F0DE0AB48AA49B0F866
:10EEE0007C0F91F87E1F06E0A748B0F8800F02E083
:10EEF000A548B0F8840F00EB014080B270472DE9BF
:10EF0000F047A24CDFF88882DFF88892A36DDFF823
:10EF100088A233F8021BA365188801F47F4242EAF5
:10EF200010254FF6FF7202EA0026CAB2226632436B
:10EF30004AF28746A91BB54270D041DC274648F209
:10EF4000826C796E3F8AA5EB0C06654568D01FDCA4
:10EF500048F28A48A5EB080C4FF00106454556D00B
:10EF600009DC1CF1080540D0022D41D0042D48D009
:10EF7000062D72D148E0BCF1020F48D0BCF1040F5D
:10EF800045D0BCF1060F42D0BCF5FB7F65D141E016
:10EF900041F6016CA6EB0C00664566D009DC022E3A
:10EFA00045D0042E47D0062E49D0B6F5F05F54D197
:10EFB00057E0012855D0022857D003284DD150E002
:10EFC0000A2952D007DC48D2DFE801F0474B4F4B0B
:10EFD0004F4B4F4B4F4BA1F2FB1108293DD2DFE8BD
:10EFE00001F0484C565A64687276C2B2822001E041
:10EFF000C2B28420FFF747FDA06D801CA065667239
:10F000002BE0C2B28620F5E7C2B28820F2E7C2B296
:10F01000E8B2EFE7D019614A104404E025E0FFE7C9
:10F02000D01900F120209B1C0160A36515E03A4433
:10F0300002EB0800F7E73A4402EB0900F3E73A4431
:10F0400002EB0A00EFE72066E8B2C2F30522616E28
:10F05000FFF719FDA06D801CA065A06D001DA065C7
:10F060000EE41046FFF7FEFEEDE71046FFF721FF26
:10F07000E9E71046FFF7F6FE02E01046FFF719FF3A
:10F08000C2F30D0101EB400000F1202028E0104602
:10F09000FFF7E8FE02E01046FFF70BFFC2F30D0199
:10F0A00001EB400101EB08001AE01046FFF7DAFE21
:10F0B00002E01046FFF7FDFEC2F30D0101EB400137
:10F0C00001EB09000CE01046FFF7CCFE02E0104611
:10F0D000FFF7EFFEC2F30D0101EB400101EB0A0067
:10F0E000B4F8641089B20160B4E72DE9F05F274CF1
:10F0F000DFF89C90DFF89CA0A06DDFF89CB04FF487
:10F10000FD7E30F8021BA065B0F8008001F47F425C
:10F1100042EA18234FF6FF7202EA0825CAB22266B5
:10F120002A4349F28565591BAB4276D05CDC49F233
:10F130008345A3EB0501AB4247D03BDC254648F2B3
:10F14000826C696E2D8AA3EB0C070EB2634575D0F5
:10F1500026DC48F2864CA3EB0C074FF0010963450F
:10F160006DD008DC3B1D6BD0022B6AD108F0FF028A
:10F1700089B2842097E0022F61D0774561D151197F
:10F18000064A11449EE000000010002030000020DC
:10F19000001A002000300020D0370020001E002080
:10F1A000022F73D0042F72D0062F71D0B7F5606F85
:10F1B00047D1A2E005296CD008DC012969D00229D9
:10F1C00003D0032965D0042974D19AE0062973D0AD
:10F1D000A1F58071FF3970D001296FD0022969D162
:10F1E0001046FFF7D7FDD3E040F60365A1F60360B4
:10F1F000A94219D026DC40F6FE55A1F6FE50A942E0
:10F200001BD012DC032975D008DC012973D0022938
:10F2100050D11046FFF7D8FDC7E08CE004296BD031
:10F22000A1F55061FD3945D19FE0012871D0022838
:10F2300003D003286DD004283CD19AE03FE02EE0B3
:10F2400028E037E040F2FD15A0F2FD11A8426ED093
:10F250000BDC01286CD070456BD0881C6AD001286B
:10F2600028D11046FFF7CAFD92E0012972D0022989
:10F2700071D0032970D004291CD11046FFF7D8FDA6
:10F28000C2F30D0101EB4001594458E01CE01FE0BE
:10F2900022E032E008F0FF0289B2822003E008F0A9
:10F2A000FF0289B2D8B2FFF7EEFBA06D801CA0650B
:10F2B00084F80990BDE8F09F23E026E02AE0511988
:10F2C00001F120210E803EE02A4402EB0901F9E71A
:10F2D0002A4402EB0A01F5E72A4402EB0B01F1E7AD
:10F2E0002066B4F86400C2F3052281B2D8B2FFF7F9
:10F2F000CAFB27E031E029E033E01046FFF74AFD82
:10F30000EEE71046FFF760FDEAE71046FFF742FD23
:10F3100003E02AE01046FFF757FDC2F30D0101EBB1
:10F32000400000F12020B4F8641001800AE02CE0D5
:10F330001FE022E025E01046FFF746FD28E0B4F884
:10F3400064000880A06D801CA065B3E71046FFF73D
:10F3500021FD2AE022E025E02DE01046FFF71AFD0E
:10F360008EE71046FFF730FD8AE71046FFF746FDAF
:10F37000B6E71046FFF75CFDB2E71046FFF73EFD2B
:10F38000CBE71046FFF754FDC7E71046FFF750FDE7
:10F39000C2F30D0101EB40014944D0E71046FFF7ED
:10F3A0002DFD02E01046FFF743FDC2F30D0101EB16
:10F3B00040015144C3E71046FFF720FD60E72DE907
:10F3C000FF5FF84C49F28467F74DA16DDFF8DC93DD
:10F3D000DFF8DCA331F8022BA16502F47F43088833
:10F3E000D2B243EA10264FF6FF7303EA00232266E7
:10F3F0001A43F31BBE4278D078DCEE4B49F2870803
:10F40000A6EB080C33F8FE7C0397DF8E02975F8F24
:10F410000197DF8F0097B3F842E0B3F846B0B3F836
:10F420004A70B3F84E3046457ED046DC234648F25B
:10F4300086681B8AA6EB080C464576D022DC48F28B
:10F44000864CA6EB0C074FF0010866456ED00DDC2C
:10F45000A6F50046803E6AD0B6F5007F67D0A6F5D7
:10F460008066023E70D0022E6FD101E1022F6DD076
:10F47000B7F5FD7F6BD0B7F5FE7F56D0B7F5FF7FB0
:10F4800063D11AE140F6FD15ACF6FD10AC452BD06A
:10F490000CDCBCF1020F7DD010F1030C7BD0BCF171
:10F4A000010F79D0BCF1020F4FD19BE1012874D03C
:10F4B000022873D0032848D117E1BCF57F7F6ED0B6
:10F4C0001FDC40F2FD15ACF2FD10AC4565D00EDC42
:10F4D00010F1040C5FD0BCF1010F5DD0BCF1020F44
:10F4E000E3D0BCF1030F30D17AE14FE130E00128E5
:10F4F00054D002287CD0032816D0B0F5FF7F24D149
:10F50000FDE040F20141ACF201408C4571D011DCCC
:10F5100010F1040C6ED0BCF1010F6CD0BCF1020FE5
:10F520006AD0BCF1030F03E0E1E0CCE0AEE097E08D
:10F530000BD108E101287BD0B0F5FD7F79D0A0F593
:10F540008070FB3801D11AE18CE09BE0A4E0A8E0D8
:10F55000984E40F6014C4436A3F601403788019797
:10F56000B7880097B6F808E0634571D04CDCA6F682
:10F570007C70B3F5206FB0F838BEB0F86CCFB0F83F
:10F58000707FB0F8746FB0F8780F3CD01DDC052B9D
:10F590005FD005E09AE0ACE0ADE093E027E0B2E0B8
:10F5A00008DC012B6FD0022B6ED0032B6DD0042B07
:10F5B0007DD107E1A3F51063FC3B18D0012B6FD080
:10F5C000022B15D0032B72D107E140F6FD38A3F6CC
:10F5D000FD35434564D010DC15F5FE7338D0012BA2
:10F5E0006FD0022B78D0A3F58073FB3B5FD179E01D
:10F5F00075E0B3E095E098E0A1E0012D75D0022D13
:10F600006ED0032D53D165E0B0F5017F69D01ADCCF
:10F6100040F2FF15A0F2FF13A8426ED00ADC0128C9
:10F6200063D0022858D0981C68D001283FD1DFE071
:10F6300098E0A0E0012B71D0022B70D0032B6FD08B
:10F64000042B34D1E8E0A0F2FD3008282FD201E0ED
:10F65000C8E0BBE0DFE800F0F0F4FEECEBEAE9E83C
:10F66000628322E0C0B2FFF792FA00F00F0003E0DD
:10F67000C0B2FFF78CFAC0B2608384F80A80A06D34
:10F68000801CA06513E085E088E097E0C0B2FFF73A
:10F690007EFAC0F30B00EFE7C0B2FFF778FAEBE7B2
:10F6A00098E0D018444A104405E0891CA165B4F9DB
:10F6B0001A0004B0FEE5008890E01A4402EB09004D
:10F6C000F9E78DE008E0D0182844F4E71A4402EB8B
:10F6D0000A00F0E7104481E00EEB02007EE004E057
:10F6E0007BE09DE00BEB020078E0B81876E098181C
:10F6F00074E00398EEE70298ECE77DE074E01046D2
:10F70000FFF748FB02E01046FFF75EFB2066C2F3FE
:10F710000520FFF73CFA00F00F0035E070E073E0E1
:10F7200076E01046FFF736FB02E01046FFF74CFB91
:10F730002066C2F30520FFF72AFAC0B224E0104683
:10F74000FFF728FB02E01046FFF73EFB2066C2F3FE
:10F750000520FFF71CFAC0F30B0015E01046FFF779
:10F7600019FB02E01046FFF72FFB2066C2F30520CD
:10F77000FFF70DFA08E01046FFF70CFB63E01046B8
:10F78000FFF722FB5FE00088608378E71046FFF711
:10F7900001FB66E01046FFF717FB62E01046FFF73B
:10F7A000F9FA6CE03000002000300020001A002040
:10F7B000D0370020381F0020001E00201046FFF721
:10F7C00003FB5CE01046FFF7E5FA65E01046FFF743
:10F7D000FBFA61E00CEB020000E0B018608364E724
:10F7E000009877E7019875E71046FFF707FB8DE76C
:10F7F0001046FFF71DFB89E71046FFF7FFFA97E772
:10F800001046FFF715FB93E71046FFF7F7FA9DE761
:10F810001046FFF70DFB99E71046FFF7EFFAA4E754
:10F820001046FFF705FBA0E733E02EE024E01FE0E1
:10F8300014E00FE004E0FFE71046FFF7DFFA02E014
:10F840001046FFF7F5FAC2F30D0101EB400000F19D
:10F85000202098E71046FFF7D1FA02E01046FFF7A4
:10F86000E7FAC2F30D0101EB400101EB09008AE761
:10F870001046FFF7C3FA02E01046FFF7D9FAC2F3C9
:10F880000D0101EB400028447DE71046FFF7B6FA72
:10F8900002E01046FFF7CCFAC2F30D0101EB400184
:10F8A00001EB0A006FE72DE9F84FF54CF74D4AF2EE
:10F8B000842CA06DDFF8CC93DFF8CC8330F8022BDA
:10F8C000A06502F47F430188D2B2226643EA112781
:10F8D0004FF6FF73B5F800E0AE8803EA0123009607
:10F8E0001A43B5F808B0AE89A7EB0C0304F16C0518
:10F8F00067455FD075DC48F28663A7EB030C9F4237
:10F900006ED032DC48F28A4CA7EB0C034FF00106B4
:10F9100067457DD017DC48F2844CA7EB0C036745A4
:10F9200077D00BDCA7F50047803F73D0B7F5007F99
:10F9300070D0A7F58067023F6DD1B8E0022B6BD085
:10F94000042BF9D1C7E0B3F5FB7F7DD006DC022B99
:10F950007BD0042B7AD0062BEED1D5E0B3F5FC7F1B
:10F9600075D0B3F5FD7FE7D1DBE0C94941F6FF185B
:10F97000ACEB0807B1F838AEB1F86C3FB1F8709F46
:10F98000B1F8741FC44572D015DC41F6FC17ACEB1E
:10F990000706BC456CD009DCBCF1020F69D016F13A
:10F9A000020C14D0BCF1010FC6D1D3E0012E15D04A
:10F9B000022EC1D1EEE0B7F5FE7F76D008DC012F34
:10F9C00074D0022F23D0A7F58077FB3FB4D1B6E0E7
:10F9D000A7F58077FD3F4BD0012FADD1D0E000E0FF
:10F9E000A2E04FF4FF77B3F5027F71D024DC40F240
:10F9F000012CA3F2012163456BD015DCBB4269D019
:10FA00000BDC012B33D0022B50D0032B94D1E2E03E
:10FA100066E052E043E076E054E0A3F58073FF3BFC
:10FA200070D0012B88D1FAE007296CD2DFE801F011
:10FA30006BF6F5F4F3F2F10040F2FF31A3F2FF3080
:10FA4000002641F6322B03E064E04FE054E063E02F
:10FA50008B4270D017DCB3F5037F6DD00ADC10F554
:10FA6000FB736AD0012B69D0022B9DD138E19CE059
:10FA70007BE05CE0A3F500730D3B75D0A3F58073CC
:10FA8000F13B91D144E143F67E6C43F2AE6A072824
:10FA9000CBD2DFE800F038F4F3F2F1F0EF002A8087
:10FAA000801CA065FFF78BFC9FE053E088E0C8B2A4
:10FAB000FFF76DF800F00F0029E0C8B2FFF767F814
:10FAC000C0B224E0C8B2FFF762F8C0F30B001EE03A
:10FAD000F3E0A8E08DE0C8B2FFF759F880B216E075
:10FAE000C8B2FFF754F8C0F3130010E0C8B2FFF734
:10FAF0004EF820F07F400AE0C8B2FFF748F820F047
:10FB0000704004E079E033E1C8B2FFF740F82860C4
:10FB1000A6722AE15F490BE002F1202211682960F8
:10FB200024E102EB090104E002EB080101E05A497B
:10FB300011440968F3E7F2E0DDE0C2E0CCE00AEB53
:10FB400002012980801CA065FFF739FC5049B1F8FB
:10FB50003A1E49E099182980801CA065FFF72FFC08
:10FB60004B49B1F86E1F3FE0C9E009EB0201298063
:10FB7000801CA065FFF723FC4549B1F8721F33E0F4
:10FB800011442980801CA065FFF719FC4049B1F899
:10FB9000761F29E00EEB02012980801CA065FFF78B
:10FBA0000EFC3B49B1F87A1F1EE00099801C1144FD
:10FBB0002980A065FFF703FC3549B1F87E1F13E0EB
:10FBC0000BEB02012980801CA065FFF7F8FB304990
:10FBD000B1F8821F08E0B1182980801CA065FFF7EA
:10FBE000EEFB2B49B1F8861F08446880A06D001F0A
:10FBF000BDE01046FFF736F902E01046FFF759F96D
:10FC00002066C2F30520FEF7C2FF00F00F00286057
:10FC1000ABE047E042E023E01EE012E00DE01046DA
:10FC2000FFF720F902E01046FFF743F92066C2F320
:10FC30000520FEF7ACFFC0B2E9E71046FFF712F966
:10FC400002E01046FFF735F92066C2F30520FEF703
:10FC50009EFFC0F30B00DAE71046FFF703F902E05E
:10FC60001046FFF726F92066C2F30520FEF78FFF46
:10FC700080B2CCE793E08EE082E06CE060E059E097
:10FC800030000020001A002000300020781F0020E3
:10FC900000100020001E0020D03700201046FFF783
:10FCA000E1F802E01046FFF704F92066C2F30520F0
:10FCB000FEF76DFFC0F31300A9E71046FFF7D2F877
:10FCC00002E01046FFF7F5F82066C2F30520FEF7C4
:10FCD0005EFF20F07F409AE71046FFF7C3F802E08E
:10FCE0001046FFF7E6F82066C2F30520FEF74FFF47
:10FCF00020F070408BE71046FFF7B4F802E01046A2
:10FD0000FFF7D7F82066C2F30520FEF740FF7EE735
:10FD10001046FFF7A7F805E000F1202052E010465A
:10FD2000FFF7C7F8C2F30D0101EB400080B2B84203
:10FD30003FD2F1E71046FFF795F804E0484441E070
:10FD40001046FFF7B6F8C2F30D0101EB400080B298
:10FD5000B8422ED2F2E71046FFF784F813E0594676
:10FD600040F64370FEF745FC2E60A06D801CA06538
:10FD7000A06D001DA0652868BDE8F88F404421E013
:10FD80001046FFF796F8C2F30D0101EB400080B278
:10FD90006045F3D3E3E71046FFF764F802E010464E
:10FDA000FFF787F8C2F30D0101EB400080B2504528
:10FDB00006D3594640F64370FEF71BFC2E60D7E78A
:10FDC000FE490844006822E72DE9F041FC4D4FF65A
:10FDD000FF77AC6D20886288237900F47F41A41DF1
:10FDE00041EA1221AC6507EA02222688C0B210431C
:10FDF00007EA0626DAB2324305F16C031E1FA1F5AD
:10FE00000047803F02D0B7F5007705D118805A80AF
:10FE1000186803F083FD1FE0A1F50642803A01D186
:10FE2000E84917E0A1F50642823A02D100F120200C
:10FE300011E0A1F50642843A01D1E3490AE0A1F5B7
:10FE40000642863A01D1E14904E0A1F50642883A2A
:10FE500005D1DA4908440068A41C3060AC653068FC
:10FE6000BDE8F0812DE9F05FD5484179C90750D050
:10FE7000FEF7D7FE0446FEF7D4FE8346FEF7D1FE1A
:10FE80008246FFF79CFA1FFA80FC0023DFF84093BC
:10FE9000D04A3AE00BEB030102EBD10001F007017D
:10FEA000077819F80110C3EBC3050F430770002151
:10FEB0005544601802EBD00600F00707367819F8B1
:10FEC00007703E420DD06F1802EBD70607F0070708
:10FED00096F8008019F8070048EA000886F80080C4
:10FEE0000DE0681802EBD006DFF8E48200F00700AE
:10FEF00008F10808377818F8000007403770491CE7
:10FF0000C9B20729D5D95B1CDBB26345C2D3BDE8B2
:10FF1000F09F816D10318165F9E72DE9F041A84C22
:10FF20006079C00732D0FFF74AFA6066FFF7DDF864
:10FF3000FFF745FA0746A06D4FF6FF76001F012533
:10FF4000A06515E0A07A01281AD006EA45002082B3
:10FF5000A06D0838A065FFF732FA6066607A012864
:10FF600011D006EA45002082FFF7BFF86D1C2DB2C4
:10FF7000BD42E7DBA06D001DA065002020826FE779
:10FF800006EA0510E3E706EA0510ECE7A06D0C3081
:10FF9000A06565E72DE9FF5FDFF8248298F805008A
:10FFA000C0075FD0FEF73DFE8B4D35F8107005EBB6
:10FFB00040004688B0F804A0FEF733FE35F8101074
:10FFC00005EB40000091B0F802B0B0F80490FEF7E5
:10FFD00028FE0446FEF725FEFF22DFF8F8E188F848
:10FFE00000200EEBD001DFF8E8810A7800F007036B
:10FFF00008F10808039318F803301A400A70431CEC
:020000040801F1
:100000000EEBD30203F0070392F800C0029318F836
:100010000330801C0CEA030C82F800C00EEBD00CFD
:1000200000F007009CF80030019018F80000E64648
:1000300003408CF8003035F81450DFF894C1BD420D
:1000400012D8654800EB4400B0F80280B0450BD8E8
:10005000B0F80480D04507D2039A08781CF8022033
:1000600010430870BDE8FF9F5B48BD4215D300EB0D
:1000700044077988B14210D351450ED3009EB54252
:100080000BD8594509D8BE884E4506D80299107834
:100090001CF8011008431070E4E700998D42E1D389
:1000A00000EB440042885A45DCD381884945D9D9C0
:1000B00001981CF8000003438EF80030D2E72DE9C8
:1000C000FC5F3F4D424F434C6879C00752D0FFF769
:1000D0007BFE0190FFF778FE0090FFF775FE8346E8
:1000E000FEF79FFDFF21297004EBD00600F0070A00
:1000F00007F10802317812F80A3019403170411CBA
:1001000004EBD10501F007092B7812F80910801CC7
:100110000B402B7004EBD00400F00708217812F894
:100120000800014021705946019803F00AFD06D2EB
:10013000307817F80A1008433070BDE8FC9F594624
:10014000019803F003FC0AD85846009903F0FEFB1F
:1001500005D8287817F8091008432870EDE75946A4
:10016000009803F0F3FBE8D2217817F80800014368
:100170002170E2E7A86D2030A865DEE72DE9F047A1
:100180000F4E7079C00768D0FFF78DFB8246FFF7EE
:100190008AFB0546FFF787FB0446FEF742FDFF2179
:1001A0003170C1170B4E00EB517206EBE20322F0E7
:1001B00007021978A0EB0209054F0FE0D0370020A5
:1001C00030000020001E0020001A00200030002017
:1001D000DE5F00080010002000100020083719F82A
:1001E000072011401970411CCA1701EB527806EB29
:1001F000E80228F00708A1EB080892F800C018F8F8
:1002000007100CEA010C811C82F800C04FEAE17C67
:1002100001EB5C7C06EBEC01801C2CF0070CA0EBE6
:100220000C000E78C75D3E40FE4F0E70A24506DD05
:10023000187819F8071008431870BDE8F087AC4229
:1002400005DC107818F8071008431070F5E7A54290
:10025000F3DAC05D06430E70EFE7B06D2030B06595
:10026000EBE72DE9F047F04E7079C0075AD0FFF761
:10027000A6F88246FFF7A3F80546FFF7A0F8044664
:10028000FEF7CFFC01B2FF203070C817E74E01EB3C
:10029000507206EBE203E34F22F00702A1EB0209E2
:1002A0000837187819F8072010401870481CC21732
:1002B00000EB527806EBE8004A1C28F00708A2EB96
:1002C000080890F800C018F807200CEA020C8A1CF5
:1002D00080F800C04FEAE27C02EB5C7C06EBEC02AB
:1002E000891C2CF0070CA1EB0C011678CF5DDFF810
:1002F00034C33E401670A24505DD187819F80C107D
:100300000843187099E7AC4205DC017818F80C2016
:100310001143017091E7A5428FDA11F80C000643F2
:1003200016708AE7B06D1030B06586E72DE9FC5F86
:10033000DFF8F48298F80500C00779D0FFF73FF89E
:1003400087B2FFF73CF886B2FFF739F885B2FEF7BF
:1003500068FC0446FEF765FCFF2288F80020DFF801
:10036000CC92DFF8C08209EBD00200F007031178CD
:1003700008F10808019318F8033019401170411C66
:1003800009EBD10301F0070193F800C0009118F8C0
:100390000110801C0CEA010C83F800C009EBD001AD
:1003A00000F0070E91F800C018F80E0089460CEA1C
:1003B000000C81F800C09E49E246DFF868C231F8BF
:1003C0001400B84210D801EB440BBBF80280B045D2
:1003D0000AD8BBF80480A84506D2019910781CF809
:1003E000011008431070A8E6B8420FD101EB440297
:1003F000B2F80280B04509D19288AA4206D100998C
:1004000018781CF801100843187096E6B842EAD331
:1004100001EB44004188B142E5D38088A842E2D98B
:100420001CF80E104AEA010089F8000085E6FFE793
:10043000D8F858101431C8F858107EE62DE9F05F4E
:10044000794CDFF8E081794D6079C0075DD0FFF726
:10045000BBFCE062FFF7B8FC2063FEF7E2FB01B2F1
:10046000FF202070C81701EB507005EBE00720F06B
:100470000700A1EB000B08F108023B781BF8020013
:1004800003403B70481CC31700EB537305EBE306B6
:1004900023F00703A0EB030A96F800C01AF8020045
:1004A0000CEA000C881CC31700EB537005EBE00549
:1004B000891C20F0070086F800C0A1EB00092B780A
:1004C00019F8020003402B70D4E90B0103F039FB4B
:1004D00005D238781BF808100843387017E5D4E9BE
:1004E0000B0103F0C7F905D130781AF8081008435A
:1004F00030700CE5D4E90B0103F028FAEED228782D
:1005000019F808100843287001E5A06D1830A0659F
:10051000FDE42DE9F041444C6079C00752D0FFF76B
:10052000C2F96063FFF7BFF9A063FEF77AFBFF2112
:1005300000B22170C11700EB51753C49394E01EBF7
:10054000E50325F00705A0EB050E08361A781EF81E
:1005500006502A401A70421CD51702EB557C01EB5D
:10056000EC02451C2CF0070CA5EB0C0C17781CF8C2
:1005700006502F40851C1770EF1705EB577701EBDE
:10058000E701801C27F00707C01B0D78865D35400A
:100590000D70D4E90D67234CBE4206DD18781EF8B5
:1005A000041040EA010018705AE406D110781CF8D3
:1005B000041040EA0100107052E4005D45EA0005B5
:1005C0000D704DE4A06D00F11800A06548E42DE920
:1005D000F041FDF7D4FF144C60B3FFF764F9E0631A
:1005E000FFF761F92064FEF71CFBFF2100B22170C8
:1005F000C11700EB51750D490A4E01EBE50325F0DB
:100600000705A0EB050E08361A781EF806502A409A
:100610001A70421CD51702EB557C01EBEC02451C0D
:10062000177808E0DE5F000830000020001000208E
:10063000001000202EE02CF0070CA5EB0C0C1CF891
:1006400006502F40851C1770EF1705EB577701EB0D
:10065000E701801C27F00707C01B0D78865D354039
:100660000D70D4E90F67FE4CBE4206DD18781EF807
:10067000041040EA0100187081E406D110781CF8DB
:10068000041040EA0100107079E4005D45EA0005BD
:100690000D7074E4A06D00F11800A0656FE42DE901
:1006A000F047F04C6079C00756D0FEF788FE8146CF
:1006B000FEF785FE8046FEF7B4FAFF2100B22170F6
:1006C000C11700EB5174E849E54D01EBE40324F058
:1006D0000704071B08351A787C5D00F1010C2240E5
:1006E0001A70421CD41702EB547601EBE60226F096
:1006F0000706ACEB0606147816F805C004EA0C04ED
:100700001470841C4FEAE47C04EB5C7C01EBEC018C
:10071000801C2CF0070CA0EB0C0C0C781CF80500CE
:1007200045460440DFF838830C70A94506DD18788B
:1007300017F8081040EA010018707EE506D110781D
:1007400016F8081040EA0100107076E51CF8080061
:1007500044EA00040C7070E5A06D00F10C00A06587
:100760006BE52DE9F047FDF70AFFBE4CF0B3FEF74D
:1007700026FE8146FEF723FE8046FEF752FAFF2151
:1007800000B22170C11700EB5174B749B44D01EBB1
:10079000E40324F00704071B08351A787C5D00F198
:1007A000010C22401A70421CD41702EB547601EB64
:1007B000E60226F00706ACEB0606147816F805C02C
:1007C00004EA0C041470841C4FEAE47C04EB5C7CA7
:1007D00001EBEC01801C2CF0070CA0EB0C0C0C784E
:1007E0001CF80500454604400C7000E018E0DFF8F6
:1007F0007082A94506DD187817F8081040EA010054
:1008000018701AE506D1107816F8081040EA0100B1
:10081000107012E51CF8080044EA00040C700CE5A6
:10082000A06D00F10C00A06507E570B58D4C8F4DF3
:10083000A06D2844C0F34F0001F0B1FE002860799C
:100840008B494FEAC07001D0E8B12EE068B3A06DCB
:1008500042195010C31700EB537001EBE00120F078
:100860000700C0EB62007E4A0B78805C03430B708C
:10087000FFF719F8A16D0839801CA1656066BDE815
:100880007040FEF73CBBA06D42195010C31700EB3F
:10089000537001EBE00120F00700C0EB6200704AEA
:1008A0000B780832805C03400B70A06D0830A065A7
:1008B00070BD2DE9F0476B4E7079C00752D0FEF73E
:1008C000CEF98146B06DB046001D3746B065FEF7E3
:1008D00076FD86B239780020FF290CD0D8F8581060
:1008E0001FFA89F5083904460127A1464FF6FF7A19
:1008F000C8F8581022E0002008E000BF39F91020A5
:1009000000F10100551944EBE27480B2B042F5D316
:10091000D8F858100839C8F8581014E0D8F858100A
:10092000091FC8F858100AEA0711A8F81010FEF7B6
:1009300096F9451949EB04047F1CBFB2B742EDD3C9
:10094000FF2188F800103246002328462146F4F79C
:100950005BF94446C8F86400FEF7C7FBA06D001DB4
:10096000A0656AE4B06D0C30B06566E42DE9F0472F
:100970003C494879C2070846806D6FD08946C865F2
:10098000FEF791FFC21700EB127121F00F03C51A99
:100990000911CB1701EB137323F00F03CE1A00EBF1
:1009A00012610912CB1701EB137323F00F03CF1A57
:1009B00000EB12510913CB1701EB137300EB12403C
:1009C00023F00F030014A1EB030CC21700EB12710C
:1009D00021F00F030911CC1701EB147424F00F045C
:1009E0000C1B00EB1261C31A00EB12500013C2176C
:1009F00000EB127222F00F020912801A4FEAE1781E
:100A00001C4A01EB187828F00F085043A1EB0801AD
:100A100043F60952514300EB811040F635414C43F7
:100A200040F271214B4300EB44100CEB4C0100EB06
:100A30000310C1EBCC1100EBC10007EBC70101EBC8
:100A4000071100EB810006EB860100EB4100411924
:100A5000C9F86410BDE8F047FEF751BA10300BE05A
:100A6000DE5F00083000002000100020A49FFFF788
:100A7000CD07002080969800886543E470B5FEF7A6
:100A80009EFC0546FEF7CDF80446FEF798FCFE49AD
:100A900001EB400131F8022C2A40002101E0491C01
:100AA000C9B28142FBDBF949521E0120904021F876
:100AB000140070BD2DE9FF47F34DDFF8D483903D5E
:100AC000F44C6879F44EC0074FF000076DD0FEF784
:100AD00076FC8146FEF773FCA96D11F8042BAA7011
:100AE000A965EA49B1F8181F814205DB94F8E311C2
:100AF00041F0200184F8E311002A54D194F8F21156
:100B0000890750D4317800294DD114F8A01F41F045
:100B10000101217004F24314217801F0DF012170FA
:100B200001213170DD49088009EBC900DC49000171
:100B300091FBF0F54FF40070ADF80C0003208DF838
:100B40000E0010208DF80F006D1E03A9D548F0F798
:100B5000FCF901210220F0F73EFC46464046F0F742
:100B600009FD4720ADF80000ADF80450ADF806705F
:100B7000ADF8027069463046F0F794FD0121304629
:100B8000F1F760FA012211463046F1F749F80121E8
:100B90003046F1F730F801210220F0F71CFCE07B31
:100BA00040F00800E073BDE8FF87A86D017A0C30C3
:100BB000A970A8650029F6D130780128F3D1BA4888
:100BC000F1F719F8002145464046F1F714F80121E4
:100BD0002846F1F737FA002201212846F1F720F8DC
:100BE000377014F8A00F00F0FE00207094F8520146
:100BF00000F0F70084F85201D5E72DE9F041A24C4E
:100C0000AA4D903CA06D2844C0F34F0001F0C7FCF2
:100C1000A74ED0B1607940006071A06D008820F4CB
:100C2000504001F0CAFCA0BBA06D41194810C2178A
:100C300000EB527006EBE00220F00700C0EB610011
:100C40009C491378405C034048E09A4F207B083F62
:100C5000012860794FEA40006071A06D008820F49F
:100C600050401AD001F0A9FC98B1607940F0010021
:100C70006071A06D41194810C21700EB527206EB6B
:100C8000E20022F00702C2EB61010378C95D0B4369
:100C90000370A06D801CA06586E401F08EFC002826
:100CA000F7D0208C7B4901EBD00100F007000978D8
:100CB000385C0142EDD0607940F001006071A06DB8
:100CC00041194810C21700EB527006EBE00220F009
:100CD0000700C0EB61001378C05D03431370D8E7D1
:100CE0002DE9F041684C714D903CA06D2844C0F353
:100CF0004F0001F054FC6F4F6D4E083FA8B3207BAE
:100D0000012860794FEA40006071A06D008820F4EE
:100D1000504003D001F051FC90B145E001F04DFC92
:100D2000F0BB208C5B4901EBD00100F00700097893
:100D3000385C014238D0607940F00100607121E0F8
:100D4000607940F001006071A06D41194810C21730
:100D500000EB527006EBE00220F00700C0EB6100F0
:100D600054491378405C03401DE0FFE76079400080
:100D700000F0FE006071A06D008820F4504001F08A
:100D80001CFC68B1A06D41194810C21700EB5270ED
:100D900006EBE00220F007001378C0EB610000E0F2
:100DA00002E0C05D03431370A06D801CA06503E4E6
:100DB0002DE9F041344C3D4E903CA06D3044C0F3E1
:100DC0004F0001F0ECFB0028A06D394F008820F4A3
:100DD000504014D001F0F1FB80BBA06D8119481088
:100DE000C21700EB527007EBE00220F00700C0EBE7
:100DF000610030491378405C034013701FE001F03C
:100E0000DCFBD8B1A06D81194810C21700EB5270FD
:100E100007EBE00220F00700C0EB610025491378E2
:100E20000839405C034313706079C10707D040F074
:100E300001006071A06D801CA0651DE4FFE7607972
:100E400000F0FE00F5E72DE9F0410F4C174E903C05
:100E5000A06D3044C0F34F0001F0A1FB0028A06D4D
:100E6000134F008820F4504037D001F0A6FB98BB08
:100E7000A06D81194810C21700EB527007EBE00219
:100E800020F00700137817E0C000002000100020B9
:100E90000004004000100020F1000020F2000020BB
:100EA00000A24A0400100140000C0040A49FFFF77C
:100EB000CD070020E65F0008C0EB6100FE49405C02
:100EC000034013706079C1071CD040F001006071CD
:100ED000A06D801CA065DFE614E001F06EFB88B118
:100EE000A06D81194810C21700EB527007EBE002A9
:100EF00020F00700C0EB6100EF4913780839405C2F
:100F000003431370607900F0FE00E0E770B5EB4C2E
:100F1000EB4DA06D2844C0F34F0001F040FB0028CA
:100F2000A06DE84E008820F4504014D001F045FB3D
:100F300038BBA06D41194810C21700EB527006EB88
:100F4000E00220F00700C0EB6100DB491378405C51
:100F50000340137015E001F030FB90B1A06D411912
:100F60004810C21700EB527006EBE00220F00700B9
:100F7000C0EB6100D04913780839405C034313701B
:100F800002E06079C00703D0607940F0010002E020
:100F9000607900F0FE006071A06D801CA06570BDDE
:100FA00070B5C64CC64DA06D2844C0F34F0001F08B
:100FB000F6FA0028A06DC34E008820F450401BD0E4
:100FC00001F0FBFA88B9A06D41194810C21700EB77
:100FD000527006EBE00220F00700C0EB6100B6495A
:100FE0001378405C0340137002E06079C0071AD0A8
:100FF000607940F0010019E001F0DFFA0028F4D038
:10100000A06D41194810C21700EB527006EBE002C8
:1010100020F00700C0EB6100A74913780839405C55
:1010200003431370E1E7607920F001006071A06D67
:10103000801CA06570BDA14A8023916D891C9165BB
:101040000988B3EB112F05D19F49400851F82000C2
:10105000801C90657047F0B5984C8023A26D921C5F
:10106000A2651188B3EB112F1AD1984D3E21A5F539
:10107000017300BF05EB410735F811607E8053F81E
:10108000216003EB8107491E7E6011F0FF01F1D161
:10109000617929808C4940081A6051F82000A065C8
:1010A000F0BD10B5854CA06D008820F45040FDF7D0
:1010B000A6FBA06D801CA06510BD10B57F4CA06D77
:1010C000008820F4504001F09DFAA06D801CA065BE
:1010D00010BD10B5794CA06D008820F45040FDF78C
:1010E00044FBA06D801CA06510BD10B5734CA06DB5
:1010F000008820F45040FDF798FAA06D801CA06590
:1011000010BD10B56D4CA06D008820F45040FDF767
:10111000B0FAA06D801CA06510BD684B00B5986D3D
:10112000008820F45040FDF7C9FA986D801C98653E
:1011300000BD10B5614CA06D008820F45040FDF753
:10114000D2FAA06D801CA06510BD10B55B4CA06DDF
:10115000008820F45040FDF7DBFAA06D801CA065EC
:1011600010BD10B5554CA06D008820F45040FDF71F
:10117000E5FAA06D801CA06510BD2DE9F0074F4A6F
:101180000125DFF84C81916DDFF82C91DFF844C127
:1011900011F8020B91650B78A9F1080A00EB032006
:1011A00087B2D783107A030900F00F04A54000F539
:1011B000606608EB430306F0070403F59C630CEB41
:1011C000D606C82828D311F802CF891C9165097862
:1011D00007EB0C4707EB01618FB23F49D78301EB67
:1011E0008001ADB20A68BA4204DA1B889D4301D07F
:1011F000521C0A60BA4204DA317819F8042011400E
:1012000003E031781AF8042011433170BDE8F0078B
:1012100000F51C50FDF7A9BA08EB400101F520616B
:1012200091640A88ADB2BA4204D21B889D4301D0B2
:10123000521C0A8091B2B942E3D2DDE72DE9F003F6
:101240001E49234E0127C88B334606EB400000F5AC
:101250000050DFF864800588CD83087ADFF874C019
:10126000020903EB420300F00F02974000F56062B1
:1012700002F00704A8F1080903F59C630CEBD20205
:10128000C8283AD306EB450606F500561FFA87FC38
:10129000B67805EB0645104EADB206EB8006CD8361
:1012A0003768AF4205DA1B883CEA030C01D07F1C8B
:1012B0003760CB6C1B8811E0E65F0008300000202F
:1012C000A49FFFF7CD070020240100202C0500205B
:1012D0000010002000100020E0180020AB4213781E
:1012E00003D218F80440234002E019F804402343D5
:1012F00013708A6D121D8A6519E006EB400606F52B
:101300002066CE643188BFB2A94204D21B889F43B5
:1013100001D0491C318089B2A942117803D818F84C
:101320000430194002E019F8043019431170BDE887
:10133000F00300F51C50FDF718BAF0B5FB4AFC4F5E
:10134000916DA7F1080C11F8020B91650B7800EB79
:1013500003201FFA80FEA2F81EE0107AF54B00F57C
:10136000606603EBD60506F007042B78C82819D36E
:10137000091D91650978002606EB016189B2D183C8
:10138000ED4A52F820208A4202DA395D0B4002E031
:101390001CF804100B432B70BDE8F04000F51C5006
:1013A000FDF7E3B9E54901EB400101F52061116565
:1013B00009887145ECD2E8E7F0B5DC49DF4E0B4611
:1013C000087ADB8BDB4A06EB430300F5606E03F51E
:1013D000005302EBDE05D64F1B882A78A7F1080CD4
:1013E0000EF00704C82818D306EB430606F500568E
:1013F000B67803EB0643D04E9BB2CB8356F8206001
:101400009E4202DA3B5D1A4002E01CF804301A43A7
:101410002A708A6D121D8A650FE006EB4006CB83A9
:1014200006F520664E653188994202D2395D0A4040
:1014300002E01CF804100A432A70BDE8F04000F5F1
:101440001C50FDF792B92DE9F041B84C40F2011360
:101450002146A06D8825497930F8027B04F16806A1
:10146000A7F201129F427AD064DC3D2F78D023DCB2
:10147000A7F102073B2F74D2DFE807F0E7E6E5E7C4
:10148000E6E5E4E37373E2E173E0DF73DE73DD73DB
:10149000737373737373E073737373737373DCDBDE
:1014A000DAD9D8D7D673D5D4D373D2D1D0CFCECDC5
:1014B000CCCBCAC9C8C7C600512F71D00FDCA7F169
:1014C0003E07132F4DD2DFE807F0F1F0EFEEEDEC21
:1014D000EBEAE9E8E7E6E5E4E3E2E1E0DF00762FC6
:1014E00077D014DC6A2F75D008DC522F73D0532FBD
:1014F00072D0602F71D0622F33D19CE3702F6DD0EA
:10150000712F6CD0722F6BD0732F2AD1C2E3C02FF2
:1015100067D008DC782F65D07A2F64D0822F63D013
:10152000942F1ED1E2E3ED2F5FD0EE2F5ED0F12F8E
:1015300017D1EFE3D42A5AD05ADC652A59D030DCCF
:10154000352A57D017DC112A55D00BDC022A53D08C
:10155000042A52D0062A51D00E2A02D1EFE3E2E348
:1015600040E24FE0122A4AD0142A49D0162A48D025
:10157000182A47D1F1E3552A45D008DC362A76D01F
:101580004F2A75D0512A74D0532A3BD1F3E35B2AFA
:1015900070D05D2A6FD0632A6ED0642A32D1ECE31A
:1015A0001EE3CB2A69D051DCC42A67D008DC662A46
:1015B00065D0C12A64D0C22A63D0C32A22D1F5E300
:1015C000C52A5FD0C62A5ED0C92A70D0CA2A19D1CE
:1015D000EDE367E334E30DE31EE327E335E340E3A4
:1015E0004BE388E36AE36EE37BE389E38DE3F1E3B6
:1015F00035E0F0E3F0E3DCE3A2E3C1E3AEE3E1E3F3
:10160000EBE3EBE38BE0EAE3DBE1CFE1C2E1B6E160
:10161000A9E1A3E19DE197E191E180E174E16EE14F
:1016200068E162E159E150E14AE143E121E11BE176
:1016300015E10AE1FFE0DAE0C4E0AFE0A3E0A8E0F2
:1016400094E08EE088E083E07EE079E0CC3A082AFE
:1016500065D2DFE802F0E7E6E5E4E3E2E1E0F02A64
:1016600063D034DCA2F1D702192A58D220E0E4E397
:10167000ECE3F0E3FDE3FDE3FDE3FDE3FDE3FDE388
:10168000FDE3FDE3FDE3FDE39CE289E276E26BE24C
:101690005BE251E242E237E22BE220E213E208E2AF
:1016A000FDE1EEE1DEE1D1E1BEE1B8E19FE1EBE396
:1016B000DFE802F0F7F6F5F4F3F23535F1F0EFEE8E
:1016C000EDEC3535EBEAE9E8E7E63535E500FC2AEF
:1016D0006FD00BDCA2F1F1020B2A20D2DFE802F07E
:1016E000E969E8E71F1FE6E5E4E3E20040F63F733F
:1016F000A2F63F719A4270D009DC11F1300259D044
:10170000022A6DD0142A6AD0152A08D1A2E0012934
:101710007ED002297DD0A1F56741BF397AD0022160
:1017200040F64170FCF765FF2AE0FDE33000002041
:10173000E65F000800100020E018002000100020E4
:10174000A065BDE8F041C4E4A065BDE8F041A8E4AF
:10175000A065BDE8F041B0E4A065BDE8F041FDF74B
:10176000DBB8A065BDE8F041FDF734B9A06500889D
:10177000010A862909D08E2905D1C0B200F086FF62
:10178000A06D801CA065BDE8F081C0B200F049FFEB
:10179000F6E7A065BDE8F04100F09DBFA065C90770
:1017A0000FD00088B5EB102FEDD1BDE8F041C0B2ED
:1017B00041E4FCE3A065FCF7E2FE08B1A06DF0E7B0
:1017C000A06D27E2A065C907FBD00088B5EB102FFC
:1017D000D9D1BDE8F041C0B23DE429E100E02FE0FD
:1017E000A065FCF7CCFE0028EAD0A06DEDE7FA4A30
:1017F000A2F50171107860710868A0655FF03E0085
:1018000002EB40035B8822F8103001EB80030AE012
:1018100023E130E1FEE3BCE3B6E3B0E3AAE3A4E3F3
:101820009EE398E392E35B6841F82030401E10F09D
:10183000FF00E5D1A7E7A065BDE8F041FEF72FBFA7
:10184000A065BDE8F041FEF78CBFA065BDE8F041A2
:10185000FEF75FBEA065BDE8F041FEF7B8BEA0652B
:10186000BDE8F041FEF7FDBCA065BDE8F041FEF724
:1018700085BCA065C9077DD0FDF7A1FD2BE0F0E395
:10188000F2E3F2E3F2E3F2E3F2E3F2E3F2E3E1E3C1
:10189000D6E3CEE3C3E3B9E3B3E3ADE3A7E38EE37B
:1018A00088E380E3E7E3E7E3E7E3E7E3E7E3E7E3AE
:1018B000E7E3E7E3A065C90777D0FDF7F4FF12E09F
:1018C000A065BDE8F04101F039B8A065C907D2D0E4
:1018D000FDF775FDC04360662AE1A065C907EBD03E
:1018E000FDF7E1FFC0436066D5E0A065BDE8F041CB
:1018F000FEF713BBA065BDE8F04100F0EEBFA065A8
:10190000BDE8F04100F0BCBFA065C907B3D0FDF74A
:1019100056FD0546FDF753FDA16D083909E0A065A8
:10192000C80787D0FDF7BFFF0546FDF7BCFFA16DD7
:101930001039A1656066FDF7E2FA6566ABE0A06567
:10194000BDE8F04101F05DB9A065BDE8F04101F0EE
:10195000FEB8A065BDE8F04101F07CB9A065BDE826
:10196000F041FFF703B8A065C9076ED0FDF727FD6A
:10197000054600E0E7E0FDF722FD2844ABE7A0655F
:10198000C90777D0E065FDF78EFF0546FDF78BFFB1
:101990002844A8E7A065C90757D0E065FDF70FFD0B
:1019A0000546FDF70CFD281A95E7E5E1A065C90796
:1019B000E7D0E065FDF777FF0546FDF774FF281ACD
:1019C00091E7A065C90740D0E065FDF7F8FC054642
:1019D000FDF7F5FC0446FDF742F9014605FB04F06E
:1019E0000860D0E6A065BDE8F04101F05CB9A065F3
:1019F000C90772D0E065FDF7E2FC0446FDF7DFFCA5
:101A00000546FDF70EF994FBF5F302B2734E05FBA4
:101A1000134006EB420126F812304880B3E6A06579
:101A2000BDE8F04101F066B9A065C90706D1F1E053
:101A3000A065FCF7A4FD00283FF4C2AEFDF7BFFC93
:101A4000A16D091F401CA16545E746E0A065C907D7
:101A500079D0FDF728FF401C19E0A065BDE8F041F2
:101A6000FEF7E3BEA065C9076ED000BFFDF7A7FC77
:101A7000401E59E093E0A065FCF781FD0028F5D1F8
:101A80009EE6A065C907E3D0FDF70DFF401E606626
:101A9000A06D0838A065BDE8F041FDF730BAA0653B
:101AA000C9071AD0FDF78BFC0546FDF788FC0540F9
:101AB00028E0A065C90772D0FDF7F5FE0546FDF7E1
:101AC000F2FE054039E7A065C90706D0FDF777FCAF
:101AD0000546FDF774FC2843FDE60C3052E6A06590
:101AE000C9075CD0FDF7DFFE0546FDF7DCFE0543C8
:101AF00023E7A065C907F0D0FDF761FC0546FDF7B7
:101B00005EFC4540656613E0A065C90747D0FDF758
:101B1000CAFE0546FDF7C7FE45400EE7A065C907AA
:101B200078D0FDF74CFC40426066A06D001FA065B8
:101B3000BDE8F041FDF7D9BAA065C90788D0FDF727
:101B4000B2FE4042A3E7B5E064E0A065C9079AD0C1
:101B5000FDF735FC85B2FDF732FC80B225FA00F1C5
:101B6000C0F11000854017E0A065C8073FF462AEE1
:101B7000FDF799FE0546FDF796FE1AE0A065C90738
:101B8000DCD0FDF71CFC85B2FDF719FC80B205FA2C
:101B900000F1C0F11000C5402943616634E0EDE07A
:101BA000A065C807E2D0FDF77EFE0546FDF77BFE87
:101BB0004042C5416566A06D1038A065FDF79FF9EC
:101BC000A06D88E1A065C90774D0FDF7F8FB85B268
:101BD000FDF7F5FBC54016E02C05002000100020A5
:101BE000A065C807C2D0FDF75EFE0546FDF75BFEA7
:101BF000C540DFE7A065C9075CD0FDF7E0FB85B213
:101C0000FDF7DDFB85406566A06D0838A065FDF732
:101C10006CFAD5E5001DB5E5A065C807A6D0FDF7AF
:101C200042FE0546FDF73FFE8540C3E7A065BDE8DF
:101C3000F04100F0FBBDA065BDE8F041FEF71EBF1E
:101C4000A065BDE8F041FEF734BEA065C8078DD0A1
:101C5000FDF7B5FBF3F7B8F9F3F7F8FDF4F7B8F8CB
:101C600037E1A065C8079DD0FDF71DFEF3F7ACF97D
:101C7000F3F7ECFDF4F7ACF82DE6A065C90719D031
:101C8000FDF79DFB01F04AFE306000F052FDA06DB3
:101C9000001F77E5A065C9076ED0FDF704FE01F0CF
:101CA0003DFEBCE0EF4DA065C90704D0FDF787FB02
:101CB000287068E5E9E00A212970ABE7A065BDE876
:101CC000F041FEF7CFB8A065FDF7EDFD0546FDF745
:101CD000EAFDA84202D16079C10769D114E26071BE
:101CE00051E5A065BDE8F041FEF7E4BEA065BDE8A2
:101CF000F04100F0A3BEA065BDE8F04100F02BBDAF
:101D0000A065BDE8F041FEF799BBA065BDE8F041D4
:101D1000FEF7D5B9A065C9072ED0FEF755F801F03A
:101D2000DDFD60667CE0A065C90727D0FEF74CF8B2
:101D30000446FEF749F8214601F078FC6FE02BE0FD
:101D4000A065C9071AD0FEF73FF80446FEF73CF835
:101D50000146204601F026FF61E055E0A065C90775
:101D60000CD0FEF731F80446FEF72EF80146204667
:101D700001F0BEFC53E073E085E09BE0183001E524
:101D8000A065C907FAD0FEF71FF80446FEF71CF855
:101D9000214601F00FFE42E0A065C90773D0FEF7AF
:101DA00013F801F017FCF3F751FD36E0A9E0C3E0AA
:101DB000AEE1A065C90768D0FEF706F801F08EFD18
:101DC00080B2B1E6A065C9075DD0FDF7FDFF01F067
:101DD00085FD88E5E2E075E026E001E00AE044E008
:101DE000A065C9074FD0FDF7EFFF01F0F3FBF3F754
:101DF000D5FC12E0A065C90777D0FDF7E5FF01F03B
:101E0000E9FBF3F775FC08E0A065C9076DD0FDF7A5
:101E1000DBFF01F0DFFBF3F73FFDF3F777FD306009
:101E2000BDE8F04100F085BCA065C90753D0FDF7BF
:101E3000C6FA011241EA002076E6A065C8073FF421
:101E4000F9ACFDF730FD4FEA304020E6A065BDE873
:101E5000F041FEF76BBAA065BDE8F041FEF79AB815
:101E6000A065BDE8F04100F0BABDA065BDE8F04155
:101E70000CE00DE011E015E063E047E02DE036E016
:101E80003AE048E04CE030E051E024E000F03BBEB6
:101E9000A065BDE8F04100F0F2BDA065BDE8F041ED
:101EA00000F017BEA065C90715D0FDF788FAFCF74A
:101EB00048FB0EE0A065C90717D0FDF780FAFCF7D4
:101EC00040FB10E5A065C90705D0FDF778FAFCF7DF
:101ED00047FB80B2FFE4083054E4A065C90704D092
:101EE000FDF76DFAFCF73CFBFDE410304AE4A06519
:101EF000BDE8F041FFF7F9B8A065BDE8F041FFF794
:101F000000B9A065BDE8F041FFF707B9A065BDE8DD
:101F1000F041FFF70EB9A065BDE8F041FFF715B934
:101F2000A065BDE8F04100E000E1FFF71AB9A06547
:101F3000BDE8F041FEF761BEA065BDE8F041FEF7E7
:101F4000CFBEA065BDE8F041FEF732BFA065BDE899
:101F5000F041FEF778BFA065BDE8F041FEF7D6BFBF
:101F6000A065BDE8F041FFF71BB8A065BDE8F041F2
:101F700000F00FBFA065BDE8F04100F0E6BEA0652F
:101F8000BDE8F04100F05CBFA065BDE8F04100F0A5
:101F900024BFA065BDE8F04100F09ABFA065BDE890
:101FA000F04100F071BFA065BDE8F04100E009E13B
:101FB00001F042B8A065BDE8F04101F019B8A06594
:101FC000FDF7FDF90546FDF7FAF9217B012909D056
:101FD00061794906090E617185423FF72BAC41F0EA
:101FE00001007CE685427FF725AC6079F1E0A065D1
:101FF000BDE8F04100F090BFA065BDE8F04100F001
:10200000D3BFA065BDE8F04100F0AABFA065FDF711
:10201000D6F900E0E0E00546FDF7D1F905E0A0655E
:10202000FDF741FC0546FDF73EFC85423FF453AE0B
:102030006AE0A065FDF7C3F90546FDF7C0F905E0C4
:10204000A065FDF730FC0546FDF72DFC85423FF706
:1020500042AE59E0A065FDF7B2F90546FDF7AFF9CC
:1020600017E058E0F000002045E03DE032E025E0D8
:102070001AE012E007E09BE091E089E07FE077E082
:102080006DE065E05BE0A065FDF70DFC0546FDF742
:102090000AFC8542FFF61FAE36E0A065FDF78FF91A
:1020A0000546FDF78CF905E0A065FDF7FCFB05464C
:1020B000FDF7F9FB85427FF40EAE25E0A065FDF744
:1020C0007EF90546FDF77BF985428EDC6079C10714
:1020D0001ED18AE7A065FDF7E6FB0546FDF7E3FBA9
:1020E00085427FF7F8AD0FE0A065FDF768F905467A
:1020F000FDF765F905E0A065FDF7D5FB0546FDF7A1
:10210000D2FB8542BFF6E7AD607920F00100E6E53D
:1021100040F00100E3E5A065FDF751F90546FDF744
:102120004EF909E06079C1074AD152E0A065FDF798
:10213000BAFB0546FDF7B7FB854241D0F2E7A06543
:10214000FDF73DF90546FDF73AF9854238DCE9E748
:10215000A065FDF734F90546FDF731F905E0A06506
:10216000FDF7A1FB0546FDF79EFB854228DBD9E77D
:10217000A065FDF724F90546FDF721F905E0A06506
:10218000FDF791FB0546FDF78EFB854218D1C9E7A7
:10219000A065FDF714F90546FDF711F905E0A06506
:1021A000FDF781FB0546FDF77EFB854208DDB9E7BB
:1021B000A065FDF704F90546FDF701F98542B1DB9D
:1021C0006079A5E7A065FDF76EFB0546FDF76BFBA3
:1021D000F4E700F0FE0082E5A065002020731DE416
:1021E00070B5FD4AFB480021FC4EB02443F67F65E4
:1021F00090650388B4EB132F02D1DBB246F82300BD
:10220000491C801C89B2A942F3D3906570BDF44883
:102210000021418001807047EE49EF4A10B5891EC8
:10222000002043F67E639165401C31F8024F80B276
:102230000F2C01D09842F7D3916510BD2DE9F047DE
:10224000E8480068DFF8A0C3DFF8A083E84AE94F58
:10225000E14C01260025002847D0217909200129D9
:1022600016D097F8E011092915D001F0FE0040F0D2
:10227000020087F8E001DA48A038A0F8185EE5729D
:10228000E570C2F8A0619CF80000002867D05EE10C
:10229000257187F8E0018146C2F8A051E07A58B96B
:1022A000FFF79EFFE672FFF7B7FF43F67E618842B5
:1022B00002D987F8E0912EE1E07838B997F8E0018B
:1022C00000F0F70040F0040087F8E001C148A06585
:1022D0009CF8000008B9F0F7FBFDA16D0888020A20
:1022E0005E2A72D033DC71D200E033E1DFE802F025
:1022F000E76E6E6E6E6E9B6E6E6E6E6E6E6EB46E12
:102300006E6E6E6E6E6E6E6E6E6E6E6E6E6E6E6EED
:10231000CBCBCBCBCBCBCBCBCBCBCBCBCBCBCBCB0D
:10232000D0D0D0D0D0D0D0D0D0D0D0D0D0D0D0D0AD
:10233000D5D5D5D5D5D5D5D5D5D5D5D5D5D5D5D54D
:10234000DBDBDBDBDBDBDBDBDBDBDBDBDBDB7F2AEA
:1023500073D017DCA2F15F02202A37D200E0F0E050
:10236000DFE802F0A1A6A6A6A6A6A6A6A6A6A6A6F1
:10237000A6A6A6A6A6AEAEAEAEAEAEAEAEAEAEAEA5
:10238000AEAEAEAEDC2A1FD028DCCC2A0BD012DCDD
:10239000C82A08D008DCB02A71D0C52A03D0C62AC2
:1023A00001D0C72A12D190E0C92A03D0CA2A01D08D
:1023B000CB2A0BD189E0D82A06D008DCCD2A71D0EF
:1023C000CF2A6FD0D52A01D184E06CE075E0D92AFC
:1023D00003D0DA2A7ED0DB2A6FD17BE0EC2A7ED0D4
:1023E00010DCE82A7BD006DCDD2A73D0DF2A71D02E
:1023F000E52A62D173E0E92A71D0EA2A6FD0EB2A8C
:102400005BD16CE0F12A6FD006DCED2A67D0EF2AB1
:1024100065D0F02A7CD167E0F22A65D0F32A63D038
:10242000FF2A75D165E0E071891CA1650888000A62
:10243000802803D086285FD10BE041E06079C00797
:1024400002D000F01DFE57E0891CA16500F033FEAC
:1024500052E000F041FE4FE02072891CA16508881F
:10246000000A802802D0862846D109E06079C0079A
:1024700002D0FEF782FE3FE0FEF75FFF3CE03FE068
:1024800000F061FE38E0C0F30B00FCF7CEF833E05B
:10249000C0F30B00FCF7EDF82EE0C0F30B00FCF7E7
:1024A0000DF929E011E0C0F30B00FCF71CF923E063
:1024B000C0F30B00FCF72CF91EE029E00AE022E053
:1024C000C0F30B00FCF73AF916E0C0F30B00FCF781
:1024D0004CF911E0C0F30B00FCF791F90CE0C0F3EC
:1024E0000B0000F08FF807E0C0F30B00FCF7C9F910
:1024F00002E0C0B2FCF7DDF9A06D801CA065ECE63F
:10250000891CA165E9E6C0B21C2804D00F2802D0BE
:10251000FEF799FFE1E6324AB8F80010A03AA2F8B7
:10252000181EA2F8161EA2F8141EA8F80050E67095
:1025300097F8E00100F0FB0040F0080087F8E001A8
:1025400027E0FFF764FEF0F7C3FCF0F714FE2573F5
:1025500065731EE0FFF75BFE97F8E00100F0FE00F8
:1025600040F0020087F8E0011D48A038A0F8185E8E
:10257000E572E570C2F8A0618CF80050F0F7A8FC95
:1025800025736573207920B92671A8F80050F0F7FB
:10259000F2FD1348A038A0F8025EBDE8F0871649A6
:1025A000164A01EBD00100F007000978105C0142E7
:1025B00001D001207047002070470E490F4A01EBFF
:1025C000D00100F007000978105C014218D001200A
:1025D000704700005C6000083000002024010020EB
:1025E000A010002034012242F5000020E400002069
:1025F0000080214200100020CD070020DE5F00088F
:102600000020E5E7FE494979C907E1D0FD49FE4BC5
:1026100001EBD00100F007000A78185C02400A7054
:10262000D6E7F0B5F649F74AF74D4979CB0700F5FB
:102630000C5101F0070402EBD10122D000F5C06378
:102640001E4602EBD30306F007061F78AE5D374047
:102650001F7000F5185302EBD30203F0070316783E
:10266000EB5C1E401670A5F108030A781B5D1A4347
:102670000A70E64A002102EB400000F5805001801C
:10268000F0BD08782A5D10400870F0BDF0B4DC4B56
:102690005979C9071AD0DD49DFF868C300F1E002B3
:1026A000A0F1C807002401EB400102F00705D64E57
:1026B00001F520610CEBD202372F01D821F8024B33
:1026C00059620C801178735D19401170F0BC00F5EF
:1026D0005C50FCF74AB8CA4910B44879C2070846AA
:1026E000806D23D010F8022B886500880023010A32
:1026F000C64C86290AD0882908D080290BD010BC66
:1027000041F6651140F64170FBF773BF02EB002004
:10271000C0B2002103E002EB0020C0B2E82101EBCF
:102720005000C0B224F8103010BC7047001D8865FE
:10273000FAE710B5FCF775FAB149B44A68310B886D
:1027400022F8103002EB400049884180AC48816D8E
:10275000091D816510BD2DE9F047A9484079C007E2
:1027600063D0FCF77CFAB0F80090FCF778FAB0F987
:1027700000A0FCF774FA0446FCF771FAB4F90050B3
:10278000B4F90860B4F9188095FBF6FCB4F90E6052
:10279000E7880CFB068CB4F81080B4F90A30B4F961
:1027A0000C20A6EB080666447E43A683678A04F1E4
:1027B0000E01A7EB0906E681B4F90440B1F9066001
:1027C000C4F10107664307FB0A6403FB025592FB51
:1027D000F5F624B28C805343B1F9087093FBF5F2FF
:1027E0003C44B1F90670B1F90C307F4204EB470468
:1027F000664302FB03624A81B0F90020B1F90E3052
:102800001A4447F6FE739A4201DD5A1C04E0804BDD
:102810009A4201DC038000E0028048898881C888F0
:1028200008818888C88008884880B6E670B5744DED
:102830006879C00720D0FCF7F4F90446FCF7F1F9F9
:102840002978A1B171490022844214D821F81420BA
:10285000641CA4B2F8E700BF01EBD40204F0070641
:1028600015789E5D3540641C1570A4B201E0654981
:10287000654B8442F0D970BDA86D0830A86570BD65
:102880002DE9F0415E4C6079C00722D0FDF70BF8CE
:102890006066FCF734FBFDF706F807B2A06D4FF653
:1028A000FF7608380125A0650CE0607A012811D078
:1028B00006EA85002082A06D0838A065FCF71FFBA2
:1028C0006D1C2DB2BD42F0DBA06D001DA065002087
:1028D000208284E406EA4510ECE72DE9F041484CFB
:1028E0006079C00726D0FCF76AFD6066FCF7FDFB47
:1028F000FCF765FD0646A06D4FF6FF77001F01252A
:10290000A0650CE0607A012811D007EA450020821A
:10291000A06D001FA065FCF7E8FB6D1C2DB2B54251
:10292000F0DBA06D001DA0650020208257E407EABF
:102930000510ECE7A06D0C30A06550E42DE9F047E0
:102940002F484179C90746D0FCF739FD87B2FCF71B
:1029500036FD84B2FCF733FD86B2FCF762F905461A
:10296000FCF72DFD264980B2743131F81430B7FBE5
:10297000F3F203FB12770022244B1CE0641EA4B286
:10298000401E31F814C080B2B7FBFCF931F810805A
:10299000E24609FB08FC33F81580012C4CEA080CD0
:1029A0001FFA8CFC23F815C001D1012806D00AFBC0
:1029B0001977521C92B2B242E0D3EEE5B1F8028030
:1029C00007F00F0202FB08F242EA0C0223F815207E
:1029D000721C92B2EDE7816D14318165DDE570B551
:1029E00007484079C00728D0FCF71BF90546FCF7DB
:1029F00018F90446FCF715F9044931F8152009E0E7
:102A00003000002000100020E65F000800100020C9
:102A10000080FFFF31F814301A4421F8102001EB38
:102A2000450201EB440355885C8801EB40002C44CF
:102A3000448091889A881144818070BDF94810B50E
:102A40004179C90717D0FCF7ECF8C11700EB5173B7
:102A5000F54901EBE30223F00703C01AF34B1178A9
:102A6000C35C194204D0F14B0833C05C014000E064
:102A70001943117010BD816D091D816510BDE948B4
:102A800010B54179C90720D0FCF7CBF8E849B1F877
:102A9000242E21F810200A4601EB4000B2F8222E25
:102AA0004280B1F8201E8180E149B1F81E1EC1802C
:102AB000DF49B1F81C1E0181DD49B1F81A1E4181C0
:102AC000DB49B1F8261E818110BD816D091D81652C
:102AD00010BD1CB5D3484179C90710D0FCF7A1F847
:102AE000D34C04EB40018A7A0B7ACDE900328B7922
:102AF0000A79897834F81000F1F7F5FD1CBD816D75
:102B0000091D81651CBD70B5C6484079C0071DD040
:102B1000FCF787F80546FCF784F80446FCF781F8D3
:102B2000C34931F8152031F81430D21A21F8102099
:102B300001EB450201EB440355885C8801EB400042
:102B40002C1B448091889A88891A818070BD2DE958
:102B5000F047B4494879C2070846806D4ED089468F
:102B6000C865FCF7A0FE0A2190FBF1F292FBF1F49C
:102B700001FB120301FB1422642490FBF4F494FB88
:102B8000F1F501FB15444FF47A7590FBF5F595FBD3
:102B9000F1F601FB165542F2107690FBF6F696FB25
:102BA000F1F701FB1766A34F90FBF7F797FBF1FCDA
:102BB00001FB1C77DFF880C290FBFCFC9CFBF1F86A
:102BC00001FB18CCDFF8748290FBF8F090FBF1F871
:102BD00001FB18000CEB0010000600EB075000EBA7
:102BE000064000EB053000EB042000EB0210C1189A
:102BF000C9F86410BDE8F047FCF781B9103088656A
:102C0000CBE470B5874C6079C1072046806D1ED03B
:102C1000E065FCF7D4FB4FF47A7390FBF3F21103F9
:102C200003FB1202642592FBF5F341EA032005FB46
:102C300013210A2391FBF3F240EA021003FB121165
:102C400000B208436066BDE87040FCF74EBA083039
:102C5000A06570BD10B5734C6079C1072046806DCA
:102C60001ED0E065FCF7ABFBC0F303314FF47A7282
:102C70005143C0F3032202EBC20303EB021201EB48
:102C80008201C0F3031202EB820201EB420100F069
:102C90000F00084400B26066BDE81040FCF725BA9A
:102CA0000830A06510BD70B55E4C6079C0071DD0BE
:102CB000FCF7F9FD0646FCF7F6FD464304F18805EE
:102CC000F017C5E90060FBF7ACFFA16D00B2091D6C
:102CD000A16557492A8821F8102001EB40006A8835
:102CE0004280A9888180E988C18070BDA06D1830BC
:102CF000A06570BD70B54B4C6079C00721D0FCF762
:102D0000D2FD06B2FCF7CFFD00B296FBF0F100FB5E
:102D1000116004F16C052E1D29603060FBF781FF06
:102D2000A16D00B2091DA16541492A8821F8102032
:102D300001EB40006A884280318881807188C180BF
:102D400070BDA06D1830A06570BD10B5FCF7ABFD6F
:102D50000446FCF7A8FD33490A7B012A4A794FEA69
:102D600042624FEA12624A7102D084420DD010BD15
:102D70008442FCD1088C2C4B2C4C03EBD00300F08C
:102D800007001B78205C0342F1D042F0010048713B
:102D900010BD10B5FCF713FB0446FCF710FB2149EE
:102DA0000A7B012A4A794FEA42624FEA12624A716B
:102DB00002D084420DD010BD8442FCD1088C1A4B45
:102DC0001A4C03EBD00300F007001B78205C034291
:102DD000F1D042F00100487110BD10B5FCF763FD61
:102DE0000446FCF760FD0F490A7B012A4A794FEA45
:102DF00042624FEA12624A7102D084420DDB10BD7A
:102E00008442FCDD088C084B084C03EBD00300F037
:102E100007001B78205C0342F1D042F001004871AA
:102E200010BD00003000002000100020DE5F000810
:102E300000100020A086010040420F0080969800FC
:102E400010B5FCF7BCFA0446FCF7B9FACE490A7B88
:102E5000012A4A794FEA42624FEA12624A7102D06D
:102E600084420DDBDCE78442DADD088CC74BC84CBA
:102E700003EBD00300F007001B78205C0342CFD0A7
:102E800042F001004871CBE710B5FCF70CFD044699
:102E9000FCF709FDBC490A7B012A4A794FEA4262E4
:102EA0004FEA12624A7102D084420DDBB8E78442D5
:102EB000B6DA088CB54BB64C03EBD00300F0070034
:102EC0001B78205C0342ABD042F001004871A7E7B9
:102ED00010B5FCF774FA0446FCF771FAAA490A7BAC
:102EE000012A4A794FEA42624FEA12624A7102D0DD
:102EF00084420DDB94E7844292D1088CA34BA44C0E
:102F000003EBD00300F007001B78205C034287D05E
:102F100042F00100487183E710B5FCF7C4FC044699
:102F2000FCF7C1FC98490A7B012A4A794FEA4262C0
:102F30004FEA12624A7102D084420DDD70E784428A
:102F4000FCDC088C914B924C03EBD00300F00700A3
:102F50001B78205C0342F1D042F0010048715FE72A
:102F600010B5FCF7A0FC0446FCF79DFC86490A7BE3
:102F7000012A4A794FEA42624FEA12624A7102D04C
:102F800084420DDA4CE78442FCDB088C7F4B804C9A
:102F900003EBD00300F007001B78205C0342F1D064
:102FA00042F0010048713BE710B5FCF708FA04460F
:102FB000FCF705FA74490A7B012A4A794FEA426212
:102FC0004FEA12624A7102D084420DDA28E7844245
:102FD000FCDB088C6D4B6E4C03EBD00300F007005C
:102FE0001B78205C0342F1D042F00100487117E7E2
:102FF00010B5FCF758FC0446FCF755FC62490A7B07
:10300000012A4A794FEA42624FEA12624A7102D0BB
:1030100084420DD104E78442FCD0088C5B4B5C4CAD
:1030200003EBD00300F007001B78205C0342F1D0D3
:1030300042F001004871F3E610B5FCF7C0F9044610
:10304000FCF7BDF950490A7B012A4A794FEA4262EE
:103050004FEA12624A7102D084420DD1E0E6844206
:10306000FCD0088C494B4A4C03EBD00300F007001E
:103070001B78205C0342F1D042F001004871CFE69A
:1030800010B5414CA06D10F8021BA065007801EB53
:103090000022A2833F49E07901EB400101F5905104
:1030A00061640A80EFF787FAE079BDE8104000F527
:1030B000B050FBF75ABB10B5334CE079EFF7B5FAD7
:1030C000E07900F5B050FBF750FBE079BDE8104027
:1030D00000F5C060FBF749BB10B52B4CA16D11F892
:1030E000020BC0F34600A083A16509880A0A862A5C
:1030F00002D0882A0AD103E0C9B200EBC11004E073
:10310000C9B200EBC11000F57A70A0836079C007E6
:1031100016D02049A08B01EB400000F5005002883A
:10312000E07901EB400101F58051A1F80022EFF7B1
:1031300042FAE079BDE8104000F5B050FBF715BB4E
:10314000BDE81040B7E71048826D12F8021BC1F3CA
:103150004601C18382651288130A862B02D0882B10
:103160000AD103E0D2B201EBC21104E0D2B201EB0A
:10317000C21101F57A71C1834079C00701D0FEF711
:103180005DB8FEF719B900003000002000100020E3
:10319000DE5F0008001000200EF1020E2EF0030E7C
:1031A0005EF8046B364205D4012A43EB030515F59E
:1031B000001F12D8012841EB010C1CF5001F0CD890
:1031C0000ED14FEAD17C15F5001F0CEB4C0C0CF125
:1031D000020C08BF4CEBD37C04E04FF0080C01E07C
:1031E0004FEAD37C0CEB4C0526FA05F606F00706F1
:1031F000B6F1040C06D20EEB860CBDE870404CF024
:10320000010C6047DFE80CF0090B02024FF00041AF
:103210004FF00000A1F5002170BD194610460128AD
:1032200051EB010418BFD4F5001484BF002001F055
:10323000004170BD2DE9F04101F5801CBCF5001F77
:10324000C0F2C3804FEA115C21EA0C510CF1FD0C75
:1032500041F480115FEA5C0C0CF5C07C01D34000A6
:1032600049413DA4890241EA905187028E0E0A0C21
:10327000A45D04FB04F602FB06F6C6F14046A4FB7F
:103280000662F60D46EA422606FB06F4A4FB01237D
:103290005242C3F1404338BF5B1EA6FB02420024EA
:1032A000E6FB0324D20B42EA4446A6FB0623A1FB1D
:1032B00002E2A3FB07E4A4184FF0000252F100025F
:1032C000E3FB01426442C2F1404E38BFAEF1010E51
:1032D000A6FB04234FF00002E6FB0E32A2FB0346DE
:1032E0004FF00004B61954F10004E2FB0264A1FBA4
:1032F00006E6A4FB07E816EB08064FF0000858F1B5
:103300000008E4FB01687642C8F1405838BFA8F1D4
:103310000108A2FB06E4A3FB08E52D194FF0000409
:1033200054F10004E2FB0854A1FB05E6A7FB04E806
:1033300018EB06084FF0000656F10006E1FB048684
:1033400018F1200556F10006A809A8F11B08B109DB
:1033500008F03F08B8F10A0F40EA86601CD901EB7B
:103360000C51BDE8F08100BFFCF5EEE8E2DDD8D3FA
:10337000CFCBC7C3C0BDB9B6B4B1AEACA9A7A5A3E6
:10338000A19F9D9B9A9896959392908F8D8C8B89F7
:103390008887868584838281A0FB006800FB01F218
:1033A00008EB4208B8EB872807D5341858EB01041E
:1033B000D5D5401C51F10001D1E7341A78EB010456
:1033C000CDD4401E71F10001C9E75FEA4C0C5FEA01
:1033D0009C5C0DD105D34FF0000001F00041BDE829
:1033E000F081BDE8F04170B5FFF7D6FE6DDBFFBEA2
:1033F000BDE8F0414FF00000004970470000F87F41
:1034000010B591EA030F48BF83F0004332F5B8AA24
:10341000841A71EB030C07D212198CF0004C43EBA9
:103420000C03001B61EB0C01DFF8A4E14FEA11541F
:10343000A4EB135C1EEA430F18BF9EEA445F00F042
:10344000B08023EA6E03524221EA0451C3EB6E03BB
:1034500038BF5B1EDCF1200E25D322FA0CFE10EBE8
:103460000E0043FA0CFE41EB0E01CCF1200E03FAE4
:103470000EFE10EB0E0051F10001CCF1200E29D40C
:1034800012FA0EF201EB0451BDE8104058BF70472C
:10349000401C1CBFB2F1004F704700280CBF491CF4
:1034A00020F00100704712EB020E43EB030218BF3D
:1034B0004FF0010E4EEA4202ACF1200CDCF11E0E80
:1034C00054D943FA0CFE10EB0E0051F1FF31CCF150
:1034D0001E0ED5D50EF1010E12FA0EFE404141EB43
:1034E000010101EB445C5FEA5C5C10D910EBDE701B
:1034F00001EB045138BFBEF1004FBDE8104018BFCA
:10350000704700280CBF491C20F00100704730D2E2
:103510004FEAD42C11F5001124F400641BD0B1FA49
:1035200081F20B3AA41AA41ED2F12003914030FA82
:1035300003F31943904001EBCC71002C01EB0451D3
:10354000BDE81040A8BF704701F1C0414FF0000036
:1035500001F000417047B0FA80F310FA03F100D196
:1035600010BDE41A173C4805C90AE4E701EB045111
:1035700010BD491001EB0451BDE810404FEA300086
:1035800002E04FF0000170474A0008BF0042F8D047
:10359000B2F5001F28BF704701F000414FF0000056
:1035A00070479EEA445F07D011EA5E0FBDE8104005
:1035B00004BF002100207047BDE8104070B5FFF740
:1035C000EBFD00BF40DFF63E83F000411046704740
:1035D0000000E0FF43004FEAD30C4FEA3C0C4340AD
:1035E0001FBF40070CF1605113F0FE4F70471CF0F5
:1035F000006F03D100200CF0004170470CF0004335
:1036000043EA507010B540EACC0000F054FA00BF15
:10361000000000924FEA0001F2F7C4BC4FF00041F5
:103620004FF00000A1F500217047000090EA010F63
:1036300048BF81F0004100F1BC82421A3CBF801AB1
:1036400089184FEAD0524FF07F4C1CEA410FA2EB91
:10365000D15318BF9CEA026F00F03B804FF0004C42
:103660004CEA00204CEA012121FA03FC10EB0C0C7F
:103670001ED202F1FF325FEA1C2040EBC25038BF7D
:1036800070471CF07F0F4FEA400C18BFBCF17F4F12
:1036900038BF7047C3F12003994008BF20F00100F4
:1036A000BCF17F4F38BF7047A0F1C040F1F7A3BC19
:1036B0004FEA3C00000A40EBC25028BF1CF0FF0F4D
:1036C0004FEA400CE6D018BFBCF17F4F38BF7047BF
:1036D000EAE79CEA026F05D010EA5C0F08BF00F031
:1036E0000040704710B500F0E6F900BF64FBBE3E35
:1036F0004FF47F0C1CEAD0121EBF1CEAD11392EAD1
:103700000C0F93EA0C0F00F0858090EA010F48BF80
:1037100042F4807240F4000C41F400002CF07F4130
:1037200020F07F4000B58142A2EB03020FF2081C9B
:10373000ACEB504EC0F100009EF800E04FEA4E0E98
:1037400000FB0EFC38BF49004FEA2C1C02F5FA02C0
:103750000CFB0EF34FEACE1E4FEA112C4FEAC121AB
:103760000EEB635E42EB22420EFB0CFC4FEA1C5355
:1037700000FB03114FEA112C4FEA01310EFB0CFC48
:103780004FEADC4C00FB0C11C14228BF09184CEB7E
:1037900003335DF804EB10EB410143EBC250B2F58B
:1037A0007C0F38BF704729D512F0F00F1CBF00F115
:1037B000C04000F000407047008182838485868786
:1037C00088898B8C8D8E8F919293959697999A9CE0
:1037D0009D9FA0A2A3A5A7A8AAACAEB0B2B3B5B74F
:1037E000B9BCBEC0C2C5C7C9CCCED1D4D7D9DCDF25
:1037F000E2E6E9ECF0F3F7FAFE0000004FEA400CD5
:103800000CF1807CBCF17E4F28BF7047B0F1C04006
:10381000F1F7F1BB90EA010F0CEAD11348BF42F473
:103820008072624538BF634507D213F47F0F16D00C
:1038300080EA010000F00040704710B500F03BF94D
:10384000097EFC3E00F005B880EA010000F000406F
:10385000704780EA010000F00040F1F7CCBB12F4A1
:103860007F0F04BF0248704780EA0100F1F7C3BB35
:103870000000C07F50EA010C00F113801CF5000F1E
:1038800058BFBCF5000F01D48842704707D710F528
:10389000000F58BF11F5000F15D4884270478942B8
:1038A00070471CF5000F04D5BCF5000FF7D5814219
:1038B00070474FF0807C1CEB400F38BF1CEB410F72
:1038C00001D28142704710B500F0F5F8922449000A
:1038D0004FF000504FF08051F2F775BBC10DD1F1A0
:1038E0009E0206DB4FEA002343F0004323FA02F076
:1038F0007047004207D54FEA4001B1F1FE4F02D2B6
:103900004FF00000704710B500F0D5F849922480C0
:10391000002070476FEA20007047000010F000415F
:1039200048BF4042B0FA80F310FA03F2C3F19D039E
:103930000BD051EAC35101EB1220530638BF704738
:1039400000F1010008BF20F00100704750EA010CAF
:1039500000F113801CF5000F58BFBCF5000F01D417
:103960008842704707D710F5000F58BF11F5000FB8
:1039700015D488427047894270471CF5000F04D562
:10398000BCF5000FF7D5814270474FF0807C1CEBEF
:10399000400F38BF1CEB410F01D28142704710B578
:1039A00000F089F8922449004FF000504FF0805108
:1039B000F2F709BB4FF47F0C1CEAD0121EBF1CEAC1
:1039C000D11392EA0C0F93EA0C0F00F0478090EAB3
:1039D000010F48BF42F480724FF0004C4CEA0020C7
:1039E0004CEA012102EB0302A0FB0113A2F5000245
:1039F000002918BF43F001035B0028BF4FEA3303DF
:103A000042EB22425FEA132C4CEBC2502EBFBCEBC0
:103A1000436FB2F57C0F70474FEA036CBCF1004F67
:103A200008BF20F00100B2F57C0F38BF70470BD5FE
:103A300082F0FF0212F5803FC8BF704700F1C0401E
:103A4000D8BF00F00040704700F5000C5FEA4C0C56
:103A500048BF7047B0F1C040F1F7CDBA90EA010F0E
:103A60000CEAD11348BF42F48072624538BF634507
:103A700004D280EA010000F00040704710B500F069
:103A80001AF800BF8900013E00F007B800F009B83D
:103A90005FEA410C5FEA1C6C08D080EA0100F1F794
:103AA000AABA5FEA400C5FEA1C6CF6D14FF0004006
:103AB000A0F5800070470EF1020E2EF0030E5EF8A6
:103AC000044B244204D44FEA4102B2F17F4F11D893
:103AD0004FEA4003B3F17F4F0CD80ED14FEAD07CB0
:103AE000B2F17F4F0CEB4C0C0CF1020C08BF4CEB0D
:103AF000D17C04E04FF0080C01E04FEAD17C0CEBE4
:103B00004C0324FA03F404F00704B4F1040C06D2C5
:103B10000EEB840CBDE810404CF0010C6047DFE870
:103B20000CF0070802024FF00040A0F5800010BD25
:103B30000846420018BFD2F1807288BF00F00040F2
:103B400010BD51EA000C00F113801CF5000F58BFA6
:103B5000BCF5000F01D48142704707D711F5000F63
:103B600058BF10F5000F15D4814270478942704745
:103B70001CF5000F04D5BCF5000FF7D5884270473F
:103B80004FF0807C1CEB410F38BF1CEB400F01D283
:103B90008842704780EA010081EA000180EA010062
:103BA000FFF7FDBE90EA010F48BF81F000413FF5ED
:103BB00044AD421A04D882F00042A0EB0200114446
:103BC0004FEAD0524FF07F4C1CEA410FA2EBD15389
:103BD00018BF9CEA026F4AD04FF0004C4CEA00201C
:103BE0004CEA012121FA03FCB0EB0C0C0FD412F0CB
:103BF000FE0F36D05FEA4C001DD5001240EBC250DC
:103C000038BF70471CF03F0F18BF70470BE0A2F1A0
:103C100001025FEA1C2040EBC25038BF70471CF025
:103C20007F0F18BF7047C3F12003994014BF401E97
:103C300020F00100704780084FEA122308BF704748
:103C4000B0FA80FCA2EB0C02CCF1280C60FA0CF06C
:103C500093EA122F04BF00EBC25070474FEAC370C3
:103C60007047130A5FEADC1008BF7047F6E79CEA6A
:103C7000026F04D010EA5C0F08BF0020704710B537
:103C8000FFF719FF40DFF63E81F0004070470CF06F
:103C90000F03092B08BF082000F059800A2B0BD016
:103CA000082B18BF704708BF1CF0400F0AD04FF018
:103CB00000004FF0000170471CF0400F18BF4FF09C
:103CC000004070471CF0100F08D020F0704300F047
:103CD0007F4242EAD3014FEA4370704700F06040F0
:103CE00021F07F4242EA000201F07F4040EA727018
:103CF00070474FF0FF0C4CF4E06C1CEA11531CBFF2
:103D00009CEA030C9445C2BFDA4201EB02517047B2
:103D1000002B0DD0BCF1000F0FD0002A01F00041A4
:103D2000A4BF41F0E04141F07F614FF000007047D7
:103D300001F000414FF00000704750EA01334FF0AE
:103D40009B0C18BF4CF0806C71F436A970471CF4C2
:103D5000801F11D01CF4E02F03D06FEACC31490052
:103D600070474FF04050EFF3008222F0704242EA79
:103D7000000282F3008870474FF000007047C800CF
:103D8000F65E10001000000025001E000000FFFF7E
:103D90000000000000000000A500A500A500A5008F
:103DA000A50011080F000A0000000000000000003C
:103DB000000000000000000000003D001C000000AA
:103DC00000001400FF00D703000000000000FFFF08
:103DD000FFFFFFFFFFFFFFFFFFFFFFFFFFFF0000F1
:103DE000FFFF0000000000000000000000000000D5
:103DF000000000000000000000003B180000000070
:103E000000000000000000000000F40100000000BD
:103E100000000000000000000000000000000000A2
:103E20000000000000000000000000000000000092
:103E30000000000000000000000000000000000082
:103E40000000000000006400F65E100000000000AA
:103E50000000000000000000000000000000000062
:103E6000000000000000DC0DB63D00000000000076
:103E7000000000000000020003000000000000003D
:103E80000000000000000000000000000000000032
:103E90000000000000000000000000000000000022
:103EA0000000000000000000000000000000000012
:103EB0000000000000000000000000000000000002
:103EC00000000000000000000000000000000000F2
:103ED00000000000000000000000000000000000E2
:103EE00000000000000000000000000000000000D2
:103EF00000000000000000000000000000000000C2
:103F000000000000000000000000000000000000B1
:103F100000000000000000000000000000000000A1
:103F20000000000000000000000000000000000091
:103F30000000000000000000000000000000000081
:103F40000000000000000000000000000000000071
:103F50000000000000000000000000000000000061
:103F60000000000000000000000000000000000051
:103F700000000000000000000000000000003031E0
:103F800032333435363738394142434445460000F0
:103F90000000000000000000000000000000000021
:103FA0000000000000000000000000000000000011
:103FB0000000000000000000000000000000000001
:103FC00000000001020304050607080900000000C4
:103FD0000000000A0B0C0D0E0F0000000000000096
:103FE000C1814001C0804101C0804100C1814001C8
:103FF000C0804100C1814000C1814001C0804101B9
:10400000C0804100C1814000C1814001C0804100A9
:10401000C1814001C0804101C0804100C181400197
:10402000C0804100C1814000C1814001C080410089
:10403000C1814001C0804101C0804100C181400078
:10404000C1814001C0804101C0804100C181400167
:10405000C0804100C1814000C1814001C080410158
:10406000C0804100C1814000C1814001C080410049
:10407000C1814001C0804101C0804100C181400038
:10408000C1814001C0804101C0804100C181400127
:10409000C0804100C1814000C1814001C080410019
:1040A000C1814001C0804101C0804100C181400107
:1040B000C0804100C1814000C1814001C0804101F8
:1040C000C0804100C1814000C1814001C0804100E9
:1040D000C1814001C0804101C0804100C1814000D8
:1040E000C0C101C30302C2C60607C705C5C404CCCC
:1040F0000C0DCD0FCFCE0E0ACACB0BC90908C8D8FC
:104100001819D91BDBDA1A1EDEDF1FDD1D1CDC14BB
:10411000D4D515D71716D6D21213D311D1D010F08B
:104120003031F133F3F23236F6F737F53534F43C0B
:10413000FCFD3DFF3F3EFEFA3A3BFB39F9F83828DB
:10414000E8E929EB2B2AEAEE2E2FEF2DEDEC2CE4FB
:104150002425E527E7E62622E2E323E12120E0A06B
:104160006061A163A3A26266A6A767A56564A46C4B
:10417000ACAD6DAF6F6EAEAA6A6BAB69A9A868787B
:10418000B8B979BB7B7ABABE7E7FBF7DBDBC7CB43B
:104190007475B577B7B67672B2B373B17170B0504B
:1041A0009091519353529296565797559594549C8B
:1041B0005C5D9D5F9F9E5E5A9A9B5B99595898885B
:1041C0004849894B8B8A4A4E8E8F4F8D4D4C8C447B
:1041D00084854587474686824243834181804000EB
:1041E0004C5555555555A53F7751C1166CC156BF15
:1041F0009015CB19A001FA3EAD529C804F7E92BE25
:10420000C4B1B4BD9EEE213ED43888BEE9FAA8BD43
:1042100000004054FB21F93F3163621A61B4D03D84
:104220000000601A61B4D03D7370032E8A19A33B5D
:104230000000002E8A19A33BC14920259A837B39AF
:1042400000000000000000006E83F9A22915444E12
:10425000D15727FCC0DD34F5999562DB4190433C92
:10426000AB6351FE61C5BBDE3A6E24B7E0D24D426E
:10427000EA2E49061C92D1091CEB1DFE3EA729B16E
:10428000F53582E88444BB2E26709CE9417E5FB4FC
:1042900039D69139F43953838B5F849C3B28F9BD1F
:1042A000FF97F81F0F9805DE8B112FEF1F6D0A5A2D
:1042B000CF7E366DB709CB27663F464F2DEA5F9E0E
:1042C000C7BA27757BF1E5EBF739073DEA92528AC9
:1042D000B15FFB6B085D8D1FA6F810111111813FB6
:1042E000D561C119A0012ABF7DFEB157E31DC73EAC
:1042F000EB9C2B8AE6E55ABE7CD5CF5A3AD9E53DF0
:104300007AFE10111111C13F37D60684F464963F2E
:10431000280356C9226D6D3F0165F2F2D844433F30
:10432000A69237A0887E143F735360DBCB75F3BE33
:10433000FE41B31BBAA1AB3F93846EE9E326823FF3
:104340001583E0FEC8DB573F68108D1AF726303F13
:10435000E9A7F0320FB8123FD47ABF74702AFB3E3F
:104360008043010800000020240100005C010008D7
:10437000A444010824010020C4D4000078010008EE
:104380000204060800000000010203040102030405
:104390000607080900A24A0400000000000000000F
:1043A00001020304060708090000000000000000E5
:1043B000FF000000000000000000000000000000FE
:1043C00000000000000000000000000000000000ED
:1043D00000000000000000000000000000000000DD
:1043E00000000000000000000000000000000000CD
:1043F00000000000000000000000000000000000BD
:1044000000000000000000000000000000000000AC
:10441000000000000000000000000000000000009C
:10442000000000000100100000010010000000006A
:10443000000000000000000000000000000000007C
:104440000100030007000F001F003F007F00FF0076
:10445000FF01FF03FF07FF0FFF1FFF3FFF7FFFFF6E
:10446000000000000000000000000000000000004C
:104470000A00000001000000010000000000000030
:10448000000000000000000000000000000000002C
:104490000000000000000001040400020500030603
:0444A000010406000D
:0400000508000121CD
:00000001FF
